:020000040000FA
:0608000015EF5DF012008F
:0608080060EF45F0120054
:06082A000E0054BB0000AB
:10083000000500000600000052BB0000200500007B
:100840000200000050BB00001E0500000200000076
:100850004CBB00000E0500000400000049BB000076
:10086000150500000300000010BB0000C2010000DD
:1008700039000000BFBA0000600000005100000015
:1008800086BA0000C50B00003900000084BA0000E1
:100890001C0500000200000082BA00001A050000DA
:1008A000020000007EBA00000A05000004000000FB
:1008B00031920000FF0000000100000066BA000055
:1008C0005F0400001800000064BA00001805000072
:0408D0000200000022
:0C08D40005011F6B0A0E03015F6F606BD3
:1008E0000301000E5D6F070E5E6F19EC38F0010119
:1008F000A56BA66B0101000EA36F070EA46F5C0E23
:10090000B6EC11F0116E106A10C0E6FFE66E5B0ED9
:10091000B6EC11F0E552E7CF11F0E552E7CF10F059
:1009200001011010A16F11C0A2F1EAEC2AF005013B
:100930001E6F106E116A126A136AE868101805E1DA
:10094000115003E1125001E1135012000701016B35
:10095000026B05011F5124E10301D56B1EC5AEF1E9
:1009600065EC2CF0000901E15FD1620EB6EC11F0EC
:10097000010B03E1D2EC2CF053D10501010E1F6FE6
:10098000620EB6EC11F0020B04E00301010ED66F0B
:1009900002D00301D66B0701056B466B456B40D156
:1009A0001F0519E10301D5A305D0D2EC2CF00501F8
:1009B0001F6B3AD1D5B10DD0D56B0101000EB06FD0
:1009C000070EB16F84EC2CF0000913E10301D5830D
:1009D00010D0D5910ED0030E1F5D04E11F5101E030
:1009E00023D122D1020E1F5D04E11F5101E11CD170
:1009F0001BD10301D651080A01E1DED00F0A01E143
:100A0000C2D0010A01E1ABD0030A01E1A4D0010A7E
:100A100001E184D0070A6BE0010A4EE0030A0FE00F
:100A2000010A01E0FDD0250E0701005D03E103018D
:100A3000050EA7D00301020ED66FD581F1D0200E8E
:100A40000701005D2CE10551BBEC11F0EF6A350E9A
:100A50000301566F576B0301060E546F070E556F57
:100A6000C9EC37F0000913E13E0E0301566F576BD6
:100A7000070146510301546F556B060E5427070EAC
:100A80005523C9EC37F0000902E10301D66B0301DD
:100A9000D65101E0C4D00701056B466BC1D03A0EB8
:100AA000005D03E1006B0529466FC8EC11F001E31E
:100AB000B7D0FBEC11F0B4D03D0E0701005D14E19E
:100AC000006B0301030ED66F07010529106E116A32
:100AD000400E105C000E11580AE20529466F0529E8
:100AE000BBEC11F0EF6A03D0200E005D31E0030192
:100AF000D551020B04E1260E0701005D05E103015B
:100B0000040ED66F0701006BC8EC11F002E2FBEC9B
:100B100011F0040E0301D65D01E082D00301010E45
:100B2000DB6F070146510301D96FDA6B060ED92737
:100B3000070EDA230301060ED76F070ED86FC2D84F
:100B4000F35007010113F45002130301D66B0701A0
:100B5000466B056B65D000C748F7060E12D0610ED4
:100B60000701005D02E3270E04D0410E005D02E3A1
:100B7000070E005F300E005D100DF3CF47F7030145
:100B8000070ED66F4DD0610E0701005D02E3270E00
:100B900004D0410E005D02E3070E005F300E005DE1
:100BA0004713000E4B6F070E4C6F010E4D6F496BD4
:100BB0004A6B0301080ED66FD5811EC5A8F14AEC19
:100BC0002BF000092AE00301470EDC6F070EDD6FF2
:100BD000C9EC0DF0F3CF03F7F4CF04F70701000ED3
:100BE000D880F354000EF45404E200C7A9F156EC87
:100BF0002BF049C710F04AC711F0126A136AE8686F
:100C00001018E1E1E8681118DEE11250DCE1135040
:100C1000DAE1FCEC2BF0030102D00301D66BD583A3
:100C200005011F5101E095D607010151021149E06C
:100C300001C710F0020EEFEC11F001E0120001C745
:100C400010F0040EEFEC11F004E07DEC43F0D1EF76
:100C500043F001C710F0080EEFEC11F002E0D2EF04
:100C600043F001C710F0100EEFEC11F002E015EFA9
:100C700044F002C711F0106A010E111672EC11F067
:100C800002E0FFEF44F002C711F0106A200E1116C7
:100C900072EC11F002E031EF45F002C711F0106A7A
:100CA000080E111672EC11F002E0CCEF40F002C712
:100CB00011F0106A100E111672EC11F002E047EC00
:100CC00041F0120007014F6B506BD7C3E9FFD8C347
:100CD000EAFFEF506B0808E0D7C3E9FFD8C3EAFF8B
:100CE000EF50750801E0EAD10701010E516F0701CD
:100CF000746B756B0301730E486F070E496F010E1D
:100D00000301D7250301466F000E0301D82103011B
:100D1000476F36EC37F0000904E1F36AF46AC8EF74
:100D20000DF0D7C3E9FFD8C3EAFFEF5075080CE117
:100D3000070173510701746F756B000E070174276B
:100D4000010E0701752305D0070173510701746F68
:100D5000756B030E0301EA6AD725E96ED851EA22C2
:100D6000EF5062082CE1040E0301EA6AD725E96E10
:100D7000D851EA22EF50D00F106E010E105204E04D
:100D8000E846FE0B1006FCE10701776F74C72AF3F3
:100D900075C72BF342EC43F00701766FD9C3E9FF27
:100DA000DAC3EAFFEF50300805E10701771D0701BC
:100DB000761704D0070177510701761363D0D9C3A2
:100DC000E9FFDAC3EAFFEF50480818E10301760EA5
:100DD000486F070E496F010E0301D9250301466FC5
:100DE000000E0301DA210301476F36EC37F00009EA
:100DF00004E1F36AF46AC8EF0DF00AD0D9C3E6FF44
:100E0000DAC3E6FF92EC54F0E552E552F3CF76F701
:100E1000030E0301EA6AD725E96ED851EA22EF50A2
:100E20006D0830E10301770E486F070E496F040E1D
:100E30000301D7250301466F000E0301D8210301EA
:100E4000476F36EC37F0000904E1F36AF46AC8EF43
:100E50000DF00701771D106E10C0E6FF74C72AF36E
:100E600075C72BF342EC43F0E552E7CF10F01014B6
:100E70000701786F0701765107017715070178118F
:100E80000701766F0701110ED8807455000E755555
:100E900006E20701160E741901E1755105E107011B
:100EA0004F830701516BF3D00701150ED88074559D
:100EB000000E75550BE30701130E741901E175510E
:100EC00004E007014F8F0701516BE1D007011A0EB3
:100ED000D8807455000E755501E3D9D007011E0E58
:100EE000D8807455000E755501E3D1D00701220E4C
:100EF000D8807455000E75551BE307011F0E741939
:100F000001E1755106E00701210E741901E17551E7
:100F100007E107017651080802E30701516B02D08F
:100F20000701516B0701515102E107014F85AFD015
:100F30000701300ED8807455000E755521E3870ED9
:100F400003012A6F2B6B42EC43F0020814E1070106
:100F5000250E741901E1755104E1F36AF46AC8EFD2
:100F60000DF00701240E741901E1755104E1F36AD3
:100F7000F46AC8EF0DF007014F870701516B87D066
:100F80000701320ED8807455000E755505E3070130
:100F90004F890701516B7BD007015A0ED8807455D9
:100FA000000E755503E30701516B71D00701620E06
:100FB000D8807455000E755503E30701516B67D057
:100FC00007016F0ED8807455000E755505E30701B3
:100FD00050810701516B5BD00701750ED8807455A5
:100FE000000E755505E3070150830701516B4FD083
:100FF00007017B0ED8807455000E755505E3070177
:1010000050850701516B43D00701860ED880745577
:10101000000E755503E30701516B39D00701900E9F
:10102000D8807455000E755515E30701870E7419A5
:1010300001E1755107E107017651020802E307015A
:10104000516B02D00701516B0701515102E10701B9
:10105000508B1DD00701000E745D010E75590CE315
:1010600007010F0ED8807455010E755505E3070171
:1010700050870701516B0BD00701170ED8807455AC
:10108000010E755504E3070150890701516B0701F3
:10109000515112E1DBC310F0116A126A136A105049
:1010A00011101210131008E076C7A8FF74C72CF3B4
:1010B00075C72DF353EC43F0C3EF0DF0D7C3E9FF31
:1010C000D8C3EAFFEFCF10F0610E105C01E21BD233
:1010D000D7C3E9FFD8C3EAFFEF50670801E213D294
:1010E000D7C3E9FFD8C3EAFFEF50640807E0D7C3CE
:1010F000E9FFD8C3EAFFEF50650804E1F36AF46A38
:10110000C8EF0DF0870E03012A6F2B6B42EC43F002
:1011100002080BE1D7C3E9FFD8C3EAFFEF50630829
:1011200004E1F36AF46AC8EF0DF0D7C3E9FFD8C34E
:10113000EAFFEF509F0F07017A6F7B6B890E070163
:101140007A270F0E07017B23010E0301EA6AD725D8
:10115000E96ED851EA22EF5014E10301510E486FB5
:10116000070E496FD9C346F3DAC347F336EC37F0BD
:10117000000906E07AC7E9FF7BC7EAFF51C7EFFF26
:10118000C1D1010E0301EA6AD725E96ED851EA22DE
:10119000EF50780833E1020E0301EA6AD725E96EC1
:1011A000D851EA22EF50D00F106E010E105204E019
:1011B000E846FE0B1006FCE107017D6FD9C3E9FF8D
:1011C000DAC3EAFFEF5031080AE107017D1D106E16
:1011D0007AC7E9FF7BC7EAFF1050EF160ED0D9C3DC
:1011E000E9FFDAC3EAFFEF50300807E17AC7E9FF09
:1011F0007BC7EAFF07017D51EF1284D1010E030185
:10120000EA6AD725E96ED851EA22EF50630801E077
:1012100079D0020E0301EA6AD725E96ED851EA2295
:10122000EF50D00F07017D6F07017D51070869E37B
:10123000010E7DC7E7FFE75204E0E846FE0BE70634
:10124000FCE107017D6FD7C3E9FFD8C3EAFFEF5088
:101250009F0F07017A6F7B6B920E07017A270F0EA3
:1012600007017B23D7C3E9FFD8C3EAFFEF509F0FE5
:10127000230F03012A6F2B6B42EC43F007017C6FB5
:10128000D9C3E9FFDAC3EAFFEF5031080CE17AC7AE
:10129000E9FF7BC7EAFF07017D51EF1207017D518E
:1012A00007017C1316D0D9C3E9FFDAC3EAFFEF5078
:1012B00030080FE107017D1D07017D6F7AC7E9FF47
:1012C0007BC7EAFF07017D51EF1607017D5107013A
:1012D0007C17030E0301EA6AD725E96ED851EA228A
:1012E000EF5072080EE17CC7A8FFD7C3E9FFD8C34F
:1012F000EAFFEF509F0F230F03012C6F2D6B53EC70
:1013000043F000D1010E0301EA6AD725E96ED851F6
:10131000EA22EFCF10F0300E105C01E2F3D0010EA4
:101320000301EA6AD725E96ED851EA22EF5039085D
:1013300001E2E8D0010E0301EA6AD725E96ED8512F
:10134000EA22EF50D00F07017D6F020E0301EA6A17
:10135000D725E96ED851EA22EF500AE0020E0301C8
:10136000EA6AD725E96ED851EA22EF5072085BE1AC
:10137000010E7DC7E7FFE75204E0E846FE0BE706F3
:10138000FCE107017D6FD7C3E9FFD8C3EAFFEF5047
:101390009F0F2A0F03012A6F2B6B42EC43F00701CA
:1013A0007C6FD9C3E9FFDAC3EAFFEF50300810E1E0
:1013B00007017D1D07017D6F7AC7E9FF7BC7EAFF43
:1013C00007017D51EF1607017D5107017C1712D0EF
:1013D000D9C3E9FFDAC3EAFFEF5031080BE17AC75E
:1013E000E9FF7BC7EAFF07017D51EF1207017D513D
:1013F00007017C13020E0301EA6AD725E96ED85172
:10140000EA22EF5072080EE17CC7A8FFD7C3E9FFBC
:10141000D8C3EAFFEF509F0F2A0F03012C6F2D6BEB
:1014200053EC43F06FD0020E0301EA6AD725E96E50
:10143000D851EA22EF5070080AE0020E0301EA6A6E
:10144000D725E96ED851EA22EF506E085BE1010E14
:101450007DC7E7FFE75204E0E846FE0BE706FCE144
:1014600007017D6FD9C3E9FFDAC3EAFFEF50D00F60
:101470000701516F000E0701515D04E3070151514F
:10148000090802E20701516B020E0301EA6AD7253F
:10149000E96ED851EA22EF50700817E17AC7E9FFE8
:1014A0007BC7EAFF07017D51EF1207015151510738
:1014B000000901E0FAD707017D1D106E7AC7E9FF28
:1014C0007BC7EAFF1050EF161DD0D9C3E9FFDAC37E
:1014D000EAFFEF50310816E107017D1D106E7AC753
:1014E000E9FF7BC7EAFF1050EF1607015151510782
:1014F000000901E0FAD77AC7E9FF7BC7EAFF0701D5
:101500007D51EF1240D3D7C3E9FFD8C3EAFFEF50B4
:101510006C0801E082D1010E0301EA6AD725E96E69
:10152000D851EA22EF506B0A01E17FD0070A01E1AE
:101530007CD0020A35E00F0A1BE0030A01E06CD1FF
:10154000DBC310F0116A126A136A105011101210E6
:1015500013100DE00301080E4E6FD9C34CF3DAC32C
:101560004DF33E0E03014A6F4B6B5BEC37F054D1E9
:10157000DBC310F0116A126A136A105011101210B6
:1015800013100DE00301080E4E6FD9C34CF3DAC3FC
:101590004DF3350E03014A6F4B6B5BEC37F03CD1DA
:1015A000DBC310F0116A126A136A10501110121086
:1015B00013103AE00701010E516F0701526B0F0E35
:1015C0000701525D2AE2070151510AE00701525119
:1015D0000301EA6AD925E96EDA51EA22EFCF51F721
:1015E000070151510BE1200EA86E470E070152254D
:1015F00003012C6F2D6B53EC43F00AD051C7A8FFA9
:10160000470E0701522503012C6F2D6B53EC43F05D
:10161000D7EC45F00701522BD2D7A86A560E03012A
:101620002C6F2D6B53EC43F0F7D0D9C37FF7DAC39F
:1016300080F70701526B0701816B0701826B020E75
:101640000301EA6AD725E96ED851EA22EFCF10F0FC
:10165000300E105C15E3020E0301EA6AD725E96E2D
:10166000D851EA22EF5039080BE3020E0301EA6A6F
:10167000D725E96ED851EA22EF50D00F0701826FCB
:101680001F0E0701525D01E39FD007017FC7E9FFED
:1016900080C7EAFF7F2B000E8023EFCF7EF7070184
:1016A0007E5101E191D00701815112E15F0E0701E6
:1016B0007E5D03E10701812B0AD007015251522BB5
:1016C000EA6A530FE96E070EEA227EC7EFFF7BD06E
:1016D0000701810562E15F0E07017E5D0DE10701F3
:1016E0005251522BEA6A530FE96E070EEA227EC767
:1016F000EFFF0701816B50D0010E0301EA6AD72585
:10170000E96ED851EA22EF506C0833E10701516BC2
:1017100007017E51740A19E0160A13E0100A0DE061
:10172000140A07E0080A01E014D007010A0E516FFD
:1017300010D007010C0E516F0CD007010D0E516F28
:1017400008D00701080E516F04D00701090E516F30
:1017500000D0070151510AE007015251522BEA6AA9
:10176000530FE96E070EEA2251C7EFFF0701816BA5
:1017700013D0010E0301EA6AD725E96ED851EA2297
:10178000EF506B0809E17EC745F31BEC37F0100DF5
:10179000F3CF51F70701812B16D0020E0701815DAF
:1017A00012E17EC745F31BEC37F007015113070127
:1017B0005251522BEA6A530FE96E070EEA2251C7C3
:1017C000EFFF0701816B5CD7010E0301EA6AD725A1
:1017D000E96ED851EA22EF506C0812E1070152512C
:1017E000EA6A530FE96E070EEA22EF6A0401530E0C
:1017F0003E6F070E3F6F82C73DF41FEC4AF00BD0DF
:1018000052C73CF40401530E3A6F070E3B6F82C778
:1018100039F4EAEC49F000D0B6D1D7C3E9FFD8C318
:10182000EAFFEF506D0821E1DBC310F0116A126A84
:10183000136A105011101210131016E0D9C3E9FFEB
:10184000DAC3EAFFEF50720A01E00ED0CBEC29F0C8
:10185000FF0E986E966E956E936E000E866E846E79
:10186000836E816EFF0000D08ED1D7C3E9FFD8C34D
:10187000EAFFEF50770801E0EFD0010E0301EA6ABA
:10188000D725E96ED851EA22EF5066081CE1D9C38A
:10189000E9FFDAC3EAFFEF50D00F0701516F020EE4
:1018A0000301EA6AD725E96ED851EA22EF5072089F
:1018B00002E0000E01D0010E0301346F51C733F373
:1018C0009FEC44F0C8D0010E0301EA6AD725E96E07
:1018D000D851EA22EF50650821E10301510E486F0B
:1018E000070E496FD9C346F3DAC347F336EC37F036
:1018F000000913E0020E0301EA6AD725E96ED85108
:10190000EA22EF50720802E0000E01D0010E03013E
:10191000366F51C735F3E3EC44F09DD0010E03015F
:10192000EA6AD725E96ED851EA22EFCF10F0310EDE
:10193000105C37E3010E0301EA6AD725E96ED8513E
:10194000EA22EF5035082DE3D9C3E6FFDAC3E6FFFC
:1019500092EC54F0E552E552F3CF85F7F4CF86F7D9
:10196000020E0301EA6AD725E96ED851EA22EF5048
:10197000720802E0000E01D0010E0301316F85C72D
:101980002FF386C730F3010E0301EA6AD725E96E0B
:10199000D851EA22EF50D00F03012E6F1DEC44F016
:1019A0005AD0010E0301EA6AD725E96ED851EA221E
:1019B000EF506D0850E10701010E526F650E0301F3
:1019C0002A6F2B6B42EC43F0FE0B0701516FD9C31A
:1019D000E9FFDAC3EAFFEF50380808E13F0ECB5CBD
:1019E00004E00701526B3F0ECB6E14D0D9C3E9FF60
:1019F000DAC3EAFFEF5061080DE1CB50106E116AB7
:101A0000FF0E101801E1115003E00701526BCB6883
:101A100007015181070152510CE10301346B640E3F
:101A200003012A6F2B6B42EC43F00301336F9FECF1
:101A300044F0020E0301EA6AD725E96ED851EA2282
:101A4000EF50720808E151C7A8FF650E03012C6F23
:101A50002D6B53EC43F097D0D7C3E9FFD8C3EAFF0F
:101A6000EF50780801E08FD0D9C3E9FFDAC3EAFF6D
:101A7000EF50300802E1000E01D0010E0701876F20
:101A8000010E0301EA6AD725E96ED851EA22EF5028
:101A9000720834E1020E0301EA6AD725E96ED851D3
:101AA000EA22EF50D00F0701886F870E03012A6FDB
:101AB0002B6B42EC43F00701516F0701510509E11F
:101AC00087C723F4070188050401226F74EC51F0E5
:101AD00014D0020E0701515D10E1010E0701885D6F
:101AE0000CE307018851050808E387C7CCF207011A
:101AF00088050201CB6F2FEC35F045D0010E0301B4
:101B0000EA6AD725E96ED851EA22EF506F083BE127
:101B1000020E0301EA6AD725E96ED851EA22EF5096
:101B2000D00F0701886F870E03012A6F2B6B42ECE1
:101B300043F00701516F0701510511E1010E070143
:101B4000885D0DE307018851060809E387C725F47E
:101B5000070188050401246F8AEC51F014D0020EAD
:101B60000701515D10E1010E0701885D0CE30701DB
:101B70008851060808E387C7CEF2070188050201ED
:101B8000CD6F6DEC35F04FC7F3FF50C7F4FF00D0B9
:101B90001200E4EC11F0EF500701506F010EEB5012
:101BA000516F020EE926000EEA22EECF54F7EDCF78
:101BB00055F7E1EC11F0EF6A610E515D67E35151A9
:101BC000680864E34F6B610E515D536F070E50154B
:101BD000106E010E105204E0E846FE0B1006FCE108
:101BE0000701526F5351566F576B920E56270F0EC7
:101BF0005723C7DB09E15351566F576B890E5627A0
:101C00000F0E57234F8107D05351566F576B800EDD
:101C100056270F0E5723F00E5015536FE85004E16E
:101C2000B0DB01E185D030D0100E535D04E1A9DBBB
:101C300001E169D261D2200E535D03E1010E4F151F
:101C400006E0300E535D08E1010E4F1505E0080E69
:101C5000501501E1A1D1B5D1400E535D0EE150A761
:101C600003D04FB16BD202D04FA168D203016E0EE8
:101C7000E16FB90EE26F000E4CD2500E535D01E0E1
:101C80005DD2010E4F1554E1310E55D06B0E515DF2
:101C900003E0750E515D18E12CDB13E06B0E515D16
:101CA00005E1505103012A6F2B6B08D050510301FD
:101CB0002A6F2B6B000E2A27010E2B2342EC43F0D8
:101CC00058D00301F56B57D06C0E515D56E15005AD
:101CD00007E103015E0EE16FBA0EE26F000E19D24A
:101CE000020E505D07E103010E0EE16FBA0EE26FC6
:101CF000000E0FD2040E505D07E103011F0EE16FCD
:101D0000920EE26F000E05D250510AE1F2DA01E0C4
:101D100069D10301190EE16F920EE26F000EF9D145
:101D2000030E505D0AE150DB060EEB505CDB02E176
:101D3000300E01D0310E65DB05D0060E505D04E19A
:101D400040DB300EEF6ED2D1050E505D02E1470E42
:101D50004FD1100E505D01E2F1D15051210801E246
:101D6000EDD1100E505DEA6A000FE96E030EEA2213
:101D7000EF500301F56FF66BFAD06E0E515D01E086
:101D800082D04F6B0F0E5015106EC11C0F0B105CE4
:101D900001E24F83F00E5015536FE8500BE119DB51
:101DA00003E1542B000E5523AADAEECFF0F3EDCF6A
:101DB000F1F3C9D0100E535D06E1A1DAEECFF5F3D1
:101DC000EDCFF6F3D4D0200E535D3FE198DAEECF9D
:101DD00058F7EDCF59F7FDDA2BE158C710F059C786
:101DE00011F0CC0EAEDADCDA0301CF6F2E0ED06F1D
:101DF000CC0EA7DA02C058F703C059F702C010F0A2
:101E000003C011F00A0E87DACBDA0301D16F0A0E94
:101E100098DA06C058F707C059F706C010F007C097
:101E200011F0640E78DA300E06240301D26FD36B02
:101E30000701545194DAE5DAEF6E545190DA01E17A
:101E400055D187DAEE2AEF2276D1300E535D04E1C8
:101E5000020E4F1501E0A0D0500E535D04E1020EBA
:101E60004F1501E199D0400E535D04E1020E4F156C
:101E700001E0A7D0600E535D01E060D1020E4F1566
:101E800001E05CD19ED0770E515D01E0A1D04F6B97
:101E90000F0E50155B6F5A6BE80403E1BDCF5AF784
:101EA00005D0020E5B5D02E1BACF5AF70F0E5A154C
:101EB00001E04F87F00E5015536FF00E535D34E183
:101EC0005B5104E1CDEC44F0300F0ED1040E5B5DAC
:101ED00013E1CB50106E116AFF0E101801E1115082
:101EE00002E0000E01D0010E010803E16ADA610E82
:101EF000FCD067DA380EF9D0080E5B5D01E01ED128
:101F0000536B0F0EBD1401E053810F0EBA1401E0A4
:101F1000538353C7ECF3E0D9EECFEAF3EDCFEBF305
:101F200054C7E9F35DD9FED0535116E152DA03E10B
:101F3000542B000E55235BC732F368EC44F0F3CF0B
:101F4000F0F3F4CFF1F3C8D9EECFEEF3EDCFEFF32A
:101F500054C7EDF367D9E6D0100E535D11E15BC7AE
:101F600032F368EC44F0F3CFF5F3F4CFF6F3B4D9E1
:101F7000EECFF3F3EDCFF4F354C7F2F384D9D2D01C
:101F8000300E535D03E1080E4F1506E1500E535D10
:101F90000AE1080E4F1507E103017F0EE16FB90E4C
:101FA000E26F000EB6D0400E535D03E1080E4F15F0
:101FB00008E1600E535D01E0C1D0080E4F1501E04D
:101FC000BDD00301840EE16FB90EE26F000EA1D007
:101FD000730E515D19E18DD903E1F3D9300E85D02F
:101FE000505102E1350E04D0500501E0A7D03E0E5D
:101FF0000301E76FE86B70D9EECFE5F3EDCFE6F3C1
:1020000054C7E4F3CCD88ED0780E515D01E096D061
:102010005F6B010E616F0F0E50155C6F0F0E501548
:10202000606FF00E50155D6F870EA0D907015E6FCF
:102030005D5103E0100E5D5D31E15E050EE1B7D943
:1020400004E0E846FE0BE706FCE1106EE66EC2EC2B
:1020500051F0B2D911E0010E12D0020E5E5D12E114
:10206000A6D904E0E846FE0BE706FCE1106EE66E3A
:10207000BEEC35F0A1D902E1000E01D0010E07013E
:102080005F6F01D0616B615159E05D5104E15F51B7
:1020900028E1300E29D05F5136E02ED0200E5D5D54
:1020A00003E0300E5D5D4AE1020E5E5D12E17FD914
:1020B00004E0E846FE0BE706FCE1106EE66E23EC5A
:1020C00035F07AD902E1000E01D0010E07015F6FF1
:1020D00001D0616B615132E0200E5D5D0BE15F511B
:1020E00002E0310E01D0300E8CD9EF6E32D9EE689D
:1020F000ED6821D05F5107E00301880EE16FB90E52
:10210000E26F000E06D003018B0EE16FB90EE26F95
:10211000000EE36FE1D8EECFDFF3EDCFE0F354C76D
:10212000DEF312D8F4CF11F04FD9020EF3CFEBFF4C
:10213000030E11C0EBFF010EF36E04D00AD9EE6856
:10214000ED68F36AF46A1200DEC310F0116A126AD5
:102150000301E1511024F36EE2511120F46EE351BA
:102160001220F86EF4CFF7FFF3CFF6FF0800F5501A
:10217000DFC3E9FFE0C3EAFFEF6EDFC3E9FFE0C3BF
:10218000EAFFEF5003E1F368F4681200DE2BDE5142
:10219000106E116ADEC3F3FF11C0F4FF12000301D9
:1021A000E451E7250701626F000E0301E821AA6EE2
:1021B00062C7A9FF3F0EA616A680A850E5C3E9FF97
:1021C000E6C3EAFFEF6EA85003E1F368F46812007B
:1021D000E42BE451116AE4C3F3FF11C0F4FF1200D1
:1021E0000301E951010815E3E95103E1EC390F0B53
:1021F000EC6F0F0EEC17EC51090802E2370E01D01C
:10220000300EEC25EAC3E9FFEBC3EAFFEF6EE90508
:1022100003E1F368F4681200E929116AF36E11C052
:10222000F4FF12000301ED51030824E3030ED880EC
:10223000ED55040DF350F0C310F0F1C311F005E0BB
:10224000D89011321032E804FBE110C062F70F0E93
:10225000070162176251090802E2370E01D0300E01
:102260006225EEC3E9FFEFC3EAFFEF6E030E030141
:10227000ED5D03E1F368F4681200ED29116AF36E75
:1022800011C0F4FF12000301F25111E1CF0EE66E0E
:10229000030EE66EF5C3E6FFF6C3E6FF07EC55F066
:1022A000E552E552E552E5520301D46BF26BF2516F
:1022B00056D8F3C3E9FFF4C3EAFFEF6EF2514FD8EB
:1022C00003E1F368F4681200F22BF251116AF2C3D1
:1022D000F3FF11C0F4FF120077D8040EE926000EB8
:1022E000EA221200126A136A105011101210131011
:1022F00012006AD8060EEB50106EF3EF11F00F0EBD
:102300005015E96EEA6AD890E936EA36120EE926E7
:10231000030EEA2212001102F3CF11F01002F3CFE4
:1023200010F0F4501126CC0E0B6E0C6AF3CF06F0B1
:1023300011C007F0D0EF5CF0EE50EFCFEAFFE96E8E
:1023400012000B6E0C6A58C706F059C707F0D0EFA1
:102350005CF03AD8020EE926000EEA221200EA6A80
:10236000CF0FE96E030EEA22EF50120003012A6F2D
:102370002B6B42EF43F0EA6A060FE96E070EEA2282
:10238000120056C7E9FF57C7EAFFEF505215120077
:102390000551106E116A3F0E105C000E11581200AC
:1023A00006C010F007C011F0300E06241200010E16
:1023B00060C7E7FFE7521200E552E7CF10F01014B4
:1023C00012008ADF9CEF11F0DCC3E9FFDDC3EAFFF6
:1023D000120054C710F055C711F072EF11F010162B
:1023E000116A72EF11F0116A126A136AE850111043
:1023F0001210131012000551052BBDDF00C7EFFFAF
:0C2400001200E66EDEDFE552E75012002D
:04240C000701006B59
:102410000A0E005D2BE20051240DF3CF01F7F4CF3B
:1024200002F7000E01270A0E0223B9EC1CF00A0E77
:10243000EF6E55EC1EF0EF9055EC1EF0EF8255EC70
:102440001EF0EF8455EC1EF0EF9855EC1EF0EF9661
:10245000B9EC1CF0FFEC1DF0B9EC1CF022EC1EF006
:10246000B9EC1CF039EC1EF0002BD2D7120007019A
:10247000006B0A0E005D48E20051240DF3CF01F716
:10248000F4CF02F7000E01270A0E0223A5EC1CF080
:10249000EF500A0837E1A5EC1CF0EF6AA5EC1CF040
:1024A0000B0EB3C0EBFF0C0EB4C0EBFFA5EC1CF0A1
:1024B0000D0EEB6A0E0EEB6AA5EC1CF0EE5236EC3C
:1024C0001EF074EC1DF075EC1EF0EF8075EC1EF044
:1024D000EF96A5EC1CF033EC1CF005E1115003E184
:1024E000125001E1135008E0A5EC1CF0B3EC1CF015
:1024F000A5EC1CF0FFEC1DF075EC1EF0EF8207015F
:1025000000511200002BB5D7FE0C07016F6B6C6BEE
:102510000A0E6C5D14E26C51240DF3CF6DF7F4CF0D
:102520006EF7000E6D270A0E6E235BEC1CF0EF5069
:102530000A0803E1010E6F6F02D06C2BE9D76F51CF
:1025400001E1FE0C0501182B000E19235BEC1CF0B9
:102550000B0E18C5EBFF0C0E19C5EBFF18C510F0DC
:1025600019C511F0126A136AD880880E1054130E20
:1025700026EC1EF003E2186B040E196F5BEC1CF0E6
:1025800088EC1DF0EF905BEC1CF00D0EB7C0EBFF7C
:102590000E0EB8C0EBFF17EC1EF01A0E2AEC1CF062
:1025A00074EC1DF00A0EE66EE66AB5C0E6FFB6C032
:1025B000E6FF5BEC1CF065EC1CF00CEC1DF0000180
:1025C000020EE76F5BEC1CF0EFEC1DF05BEC1CF017
:1025D0008BEC1EF05BEC1CF0F3EC1DF05BEC1CF0E4
:1025E000F7EC1DF05BEC1CF09EEC1CF05BEC1CF0BF
:1025F000010EEF6E17EC1EF01DEC1DF007016C5183
:1026000012000001B95151EC1CF0EF50030801E039
:10261000000C010C0001BA51240DF3CF6CF7F4CF7C
:102620006DF7000E07016C270A0E6D23BEEC1CF03F
:10263000EF5003080BE0BEEC1CF0EF50020806E080
:102640006CC7F1F06DC7F2F0ADEF19F0BAC0C4F08D
:1026500092D90CEC1DF00001110EE76FBEEC1CF0DE
:10266000EFEC1DF0BEEC1CF08BEC1EF0BEEC1CF091
:10267000F3EC1DF0BEEC1CF0F7EC1DF0BEEC1CF012
:102680009EEC1CF0BEEC1CF058EC1EF079EC1DF03A
:10269000BEEC1CF0040EEF6E12000001BB51240DC5
:1026A000F3CF76F7F4CF77F7000E070176270A0EFF
:1026B00077237DEC1CF033EC1CF007E1115005E1B1
:1026C000125003E1135001E1000C7DEC1CF03EECD4
:1026D0001EF0020B01E1000C7DEC1CF02FEC1EF053
:1026E0007DEC1CF00F0EEB500001E86F0001180E9E
:1026F000E76FEFEC1DF07DEC1CF08BEC1EF07DEC39
:102700001CF0F3EC1DF07DEC1CF0F7EC1DF07DEC03
:102710001CF09EEC1CF07DEC1CF0100EC5EC1DF0C6
:10272000126A136A7DEC1CF058EC1EF042EC1DF0AE
:102730007DEC1CF088EC1DF0EF927DEC1CF088EC39
:102740001DF0EF98010C0A0E0001BC5D01E3000CC6
:10275000BC5151EC1CF0140EFBEC1DF001E1000C1F
:10276000BC5151EC1CF00F0E2AEC1CF0EFCF10F016
:1027700078EC1EF00AE1115008E1125006E1135006
:1027800004E10301AB6B17EF26F0BC5151EC1CF0D8
:102790003EEC1EF0020B01E0010E12000001BD51E3
:1027A000240DF3CF74F7F4CF75F7000E07017427EB
:1027B0000A0E7523C3EC1CF0140EFBEC1DF001E1B6
:1027C000000CC3EC1CF033EC1CF024E1115022E1AE
:1027D000125020E113501EE10301AC6B37EC26F0E0
:1027E000E66EC3EC1CF00F0E7CEC1EF0C3EC1CF08C
:1027F00033EC1CF007E1115005E1125003E11350D6
:1028000001E1000CC3EC1CF04BEC1DF0C3EC1CF020
:1028100024EC1DF0C3EC1CF088EC1DF0EF88BEC06A
:10282000ADF35BEC26F0C3EC1CF0140E2AEC1CF0AC
:10283000EE06EF5AC3EC1CF0100E2AEC1CF0EE2A48
:10284000ED22EECF10F0EDCF11F012EC1DF003E30E
:10285000BDC0BBF022DF010C0001BF51240DF3CF3E
:102860006CF7F4CF6DF7000E07016C270A0E6D238D
:1028700087EC1CF0140EFBEC1DF001E1000C87EC62
:102880001CF033EC1CF024E1115022E1125020E145
:1028900013501EE10301AC6B37EC26F0E66E87ECBB
:1028A0001CF00F0E7CEC1EF087EC1CF033EC1CF0DF
:1028B00007E1115005E1125003E1135001E1000C52
:1028C00087EC1CF04BEC1DF087EC1CF024EC1DF0A9
:1028D00068EC1EF00001C251EE24106EC351EE20D0
:1028E000116E126A136AD880CA0E1054030E26ECB9
:1028F0001EF014E2CA0E146E030E156E166A176AE5
:1029000068EC1EF0EECF18F0EFCF19F01A6A1B6AD0
:10291000E9EC1CF010C0C2F011C0C3F087EC1CF051
:1029200088EC1DF0EF88C2C0B0F3C3C0B1F3C0C0E3
:10293000AEF3C1C0AFF37CEC26F087EC1CF0140EB4
:102940002AEC1CF00001C251EE5EC351ED5A68EC56
:102950001EF0C251EE26C351ED2287EC1CF0100E82
:10296000C5EC1DF012EC1DF003E3BFC0BBF095DE1B
:102970000001C25112000001C451240DF3CF00F731
:10298000F4CF01F7000E070100270A0E012300C74C
:10299000E9FF01C7EAFF85EC1EF001E1000C06EC3F
:1029A00028F000C7E9FF01C7EAFF88EC1EF0010C20
:1029B0000001C551240DF3CF00F7F4CF01F7000E4D
:1029C000070100270A0E0123DFEC1CF085EC1EF046
:1029D0003CE0DFEC1CF03EEC1EF0040B0CE00001D0
:1029E000FC6BFD6BC5C0FBF0D7EC1BF0DFEC1CF003
:1029F00088EC1DF0EF94DFEC1CF0120EC5EC1DF01E
:102A00000001C851105CC951115808E2DFEC1CF0FC
:102A100082EC1EF0EECFC8F0EDCFC9F0DFEC1CF079
:102A2000120EFBEC1DF007E106EC28F0DFEC1CF0C9
:102A300088EC1EF00AD0C8C0B4F3C9C0B5F3C6C054
:102A4000B2F3C7C0B3F336EF27F0F36AF46A1200AB
:102A50000001CA51240DF3CF87F7F4CF88F7000E99
:102A6000070187270A0E8823896B8A6B8B6BE4EC3E
:102A70001CF085EC1EF052E0E4EC1CF03EEC1EF085
:102A8000040B0CE00001FC6BFD6BCAC0FBF0D7EC43
:102A90001BF0E4EC1CF088EC1DF0EF94E4EC1CF06F
:102AA000120EC5EC1DF00001CD51105C000E115846
:102AB00009E2E4EC1CF082EC1EF0EFCFCDF0070150
:102AC000100E896FE4EC1CF0120EFBEC1DF00AE115
:102AD00006EC28F0E4EC1CF088EC1EF0F36A100E13
:102AE000F46E1200CEC0B9F3CDC0B8F3CBC0B6F3CC
:102AF000CCC0B7F380EC27F0F3CF8AF7F4CF8BF795
:102B000013EC1EF0200EF4180BE1115009E11250E5
:102B100007E1135005E10701200E01D0300E896F47
:102B200089C78BF78AC7F3FF89C7F4FF120000013A
:102B3000CF51240DF3CF87F7F4CF88F7000E0701AC
:102B400087270A0E882307EC1DF085EC1EF02DE088
:102B500007EC1DF03EEC1EF0040B0CE00001FC6BDA
:102B6000FD6BCFC0FBF0D7EC1BF007EC1DF088EC41
:102B70001DF0EF9407EC1DF0120EFBEC1DF007E1C9
:102B800006EC28F007EC1DF088EC1EF0000C07ECBA
:102B90001DF082EC1EF0EE06EF5AFCEC26F0D0C0E1
:102BA000E9FFD1C0EAFFEF6E010C000C0A0E000134
:102BB000D25D01E3000CD25151EC1CF085EC1EF00B
:102BC00001E0010E120007017B6B6C6B0A0E6C5D5D
:102BD00001E31FD16C51240DF3CF75F7F4CF76F7D5
:102BE000000E75270A0E762338EC1CF085EC1EF0DB
:102BF00001E00CD138EC1CF03EEC1EF0100B01E0B3
:102C000005D138EC1CF0EF500A0801E1FFD038EC98
:102C10001CF0EF50000907E138EC1CF03EEC1EF010
:102C2000010B01E0F3D038EC1CF01F0E2AEC1CF075
:102C30000201EE50F95D106EEE50FA59116E38EC4B
:102C40001CF0210E2AEC1CF051EC1DF01050125C0F
:102C50001150135801E3DAD05AEC1DF001E11200D3
:102C600038EC1CF01DEC1DF038EC1CF0210E2AECA9
:102C70001CF0010ED890EE36ED36E806FBE138EC9C
:102C80001CF01E0E2AEC1CF0EF2A38EC1CF0EF5062
:102C9000090A6EE0010A64E00F0A71E0020A6FE0BF
:102CA000030A6DE0020A56E0070A1FE0010A05E088
:102CB000030A6AE10701020E60D02CEC1EF003E368
:102CC0000701120E5AD038EC1CF03EEC1EF0010B3E
:102CD00004E038EC1CF0EF6A52D00701020E7B6F63
:102CE00038EC1CF0010EEF6E4AD02CEC1EF018E30D
:102CF00038EC1CF033EC1CF005E1115003E11250EC
:102D000001E113500AE00301CD6BCE6B38EC1CF0EF
:102D100024EC1DF0ACEC29F037D00701100E2DD0BB
:102D200038EC1CF033EC1CF005E1115003E11250BB
:102D300001E1135008E038EC1CF0B3EC1CF038EC67
:102D40001CF0FFEC1DF00701110E7B6F38EC1CF03E
:102D5000040E0CD02CEC1EF012E30701010E0DD076
:102D60000701010E7B6F38EC1CF0090EEF6E0CD0E2
:102D70002CEC1EF004E30701110E7B6F05D075C724
:102D8000F1F076C7F2F0E9DA07017B513FE07BC74B
:102D900010F0100EC8EC1CF00DE038EC1CF058ECF4
:102DA0001EF0EECF77F7EECF78F7EECF79F7EFCFD3
:102DB0007AF710D038EC1CF058EC1EF0EFCF77F714
:102DC000EE2AEFCF78F7EE22EFCF79F7EE22EFCFB2
:102DD0007AF7EF220CEC1DF07BC7E7F038EC1CF023
:102DE000EFEC1DF077C7DFF078C7E0F079C7E1F0CE
:102DF0007AC7E2F038EC1CF0F3EC1DF038EC1CF074
:102E0000F7EC1DF038EC1CF09EEC1CF007016C2B6D
:102E1000DDD61200D3C0E9FFD4C0EAFF36EC1EF0C5
:102E2000EECF80F7EECF81F7EECF82F7EFCF83F7CB
:102E3000D5C0E9FFD6C0EAFFEECF84F7EECF85F725
:102E4000EECF86F7EFCF87F70701886B060E896F05
:102E5000D7C08AF7D8C08BF7D7C039F3D8C03AF3B8
:102E600010EC36F0F3CF8AF7F4CF8BF70C0E03019A
:102E7000416F426B0301800E3F6F070E406F44ECC1
:102E800036F0F3CF8DF7F4CF8EF707018D1F8E1F2D
:102E9000D7C043F3D8C044F3B0EC36F0F3CF8FF78C
:102EA000F4CF90F70701F4508D5D61E18F518E5D95
:102EB0005EE104019B6B9C6BF1EC4BF0140E030183
:102EC000B46FB56B03016C0EB26F070EB36F36ECC7
:102ED00027F000016C0EEF6F070EF06FF5D92AECAA
:102EE0001DF0106E116A140E105E000E115A10C003
:102EF00091F71050106E116AE8500001D75DD76F3E
:102F00001150D859D86F140ED75F000ED85B2AEC39
:102F10001DF004019B6F9C6BF1EC4BF0D3C0EDF006
:102F2000D4C0EEF000016C0EEB6F070EEC6F3BD9D6
:102F300007018C6F106E13EC1EF0FE0E101805E1E9
:102F4000115003E1125001E1135011E0D7C0F8F025
:102F5000D8C0F9F000016C0EF66F070EF76FD3C002
:102F6000F4F0D4C0F5F08CC7F3F02FDA010C06ECC6
:102F700028F0010C5AEC1DF003E1D7EC45F0FAD72C
:102F800056EC1DF00DE111500BE1125009E1135008
:102F900007E10301010EAC6F37EC26F00001E86F8A
:102FA00056EC1DF007E1115005E1125003E11350FA
:102FB00001E11200140EF6EC1CF0DBC048F7DCC097
:102FC00049F7DDC04AF7DEC04BF7DFC04CF7E0C081
:102FD0004DF7E1C04EF7E2C04FF7E3C050F7E4C051
:102FE00051F7E5C052F7E6C053F7070154915493E7
:102FF00054955497E7C055F718EC28F0F3CF56F7DF
:10300000F4CF57F7F3CF10F0F4CF11F0126A136A30
:10301000000EF35C040EF458000E1258000E135804
:1030200005E30701566B040E576F0ED00701360EED
:10303000D8805655000E575505E2360E565F000EE5
:10304000575B02D0566B576B586B596B5A6B5B6B67
:103050000001480EEF6F070EF06F36D9140E000115
:10306000E927000EEA23E7C010F0020EC8EC1CF0BE
:103070000EE0040EE927000EEA230701020E5C6F42
:10308000040E5D6F5E6F5F6B5499548B03D0070124
:103090005489549B548D549F00C360F701C361F75A
:1030A00002C362F703C363F7D9C0E9FFDAC0EAFFDE
:1030B00036EC1EF0EECF64F7EECF65F7EECF66F795
:1030C000EFCF67F7686B060E696FE9C06AF7EAC071
:1030D0006BF7E9C039F3EAC03AF310EC36F0F3CFFE
:1030E0006AF7F4CF6BF70C0E0301416F426B0301DB
:1030F000600E3F6F070E406F44EC36F0F3CF58F789
:10310000F4CF59F70701581F591F58C746F759C739
:1031100047F7E9C099F4EAC09AF40401060E986FE3
:10312000D9C096F4DAC097F482EC4BF0140E030188
:10313000B06FB16B0301480EAE6F070EAF6F7CEC42
:1031400026F0E7C010F0020EC8EC1CF00BE0040EF5
:103150000301B06FB16B03015C0EAE6F070EAF6F72
:103160007CEC26F0140EF6EC1CF0E9C043F3EAC048
:1031700044F3B0EC36F0F3CF46F7F4CF47F7240E24
:10318000F6EC1CF047C7ADF35BEC26F046C7ADF399
:103190005BEC26F00301CD6BCE6BE8C0CCF321ECE9
:1031A0002AF0ACEF29F00701FE0E036F026B0A0E46
:1031B000025D51E2025134EC1DF0AEDBEF500A0823
:1031C00047E0AADB0B0EC5EC1DF07EEC1DF0020EF5
:1031D00041DB51EC1DF000011250101839E1135081
:1031E000111836E199DBEF50000902E102C703F73D
:1031F00093DB0D0EC5EC1DF07EEC1DF051EC1DF0C7
:103200001250101825E11350111822E1EDC0E9FF0A
:10321000EEC0EAFF36EC1EF0EECF14F0EECF15F064
:10322000EECF16F0EFCF17F077DBEE5236EC1EF054
:10323000EE5014180DE1EE5015180AE1EE50161874
:1032400007E1EE50171804E103E1070102511200F3
:103250000701022BACD703C710F013EC1EF0FE0ED3
:10326000101807E1115005E1125003E1135001E17C
:10327000FE0C035134EC1DF00A0EE66EE66AEDC05A
:10328000E6FFEEC0E6FF48DB20DB12507EEC1DF0CF
:1032900039DB42DB61EC1DF03FDB88EC1EF03CDBF0
:1032A000E2DA05E1115003E1125001E1135005E0AB
:1032B00033DB59DB31DBFFEC1DF02EDB88EC1DF03E
:1032C000EF82070103511200DDDAEFCF07F76FEC51
:1032D0001EF0D4DBD7DAD6EC1DF0020EE7EC1DF0C1
:1032E000020EADEC1DF0020EECEC1DF0020E7FECB8
:1032F0001EF0040EB0EC1DF0040E1CEC1EF0080EC7
:10330000B0EC1DF0080E1CEC1EF00E0EE7EC1DF0EC
:103310000E0EADEC1DF00E0EECEC1DF00E0E7FEC63
:103320001EF0100EE7EC1DF0100EADEC1DF0100EAF
:10333000ECEC1DF0100E7FEC1EF0120EE7EC1DF011
:10334000120EADEC1DF0120EECEC1DF082EC1EF036
:10335000010E80DA07C7EFFF1200B2DA84DA05E166
:10336000115003E1125001E1135008E0A9DAFBDA31
:10337000A7DAFFEC1DF0A4DACBDBEF82A1DAEE5284
:1033800036EC1EF0B1DB9CDA0D0EEB6A0E0EEB6A2A
:1033900097DA85EC1EF002E006EC28F091DA88EC72
:1033A0001EF08EDA22EC1EF08BDAB2DBEF9888DAB0
:1033B0003EEC1EF0010B03E083DAEF6A03D080DA03
:1033C0000A0EEF6E7DDA39EF1EF00001F351240D85
:1033D000F3CFB6F7F4CFB7F7000E0701B6270A0E02
:1033E000B723F8C0B1F0F9C0B2F0B86B37DA1E0EEF
:1033F00031DAEF6A33DA21DB31DA22EC1EF083DBDB
:10340000040B0EE006EC28F029DA3EEC1EF0010B6E
:1034100002E0000E01D0010EE66E20DA3EEF1DF054
:1034200099DBF1DB0E0E16DAEECF14F0EFCF15F0CC
:10343000166A176A22DA080E0DDAEE50AA5D186EC7
:10344000EE50AB59196EEE50AC591A6EEE50AD59A4
:103450001B6EBFDA03DA100EFDD9EECF1CF0EFCFF2
:103460001DF01E6A1F6A1C50105CA66F1D5011587B
:10347000A76F1E501258A86F1F501358A96F800EC7
:10348000A91506E0EBD9140EEB6A150EEB6A07D00E
:10349000E5D9140EA6C7EBFF150EA7C7EBFF6CEC22
:1034A0001EF0010820E12FDB020B06E151EC1EF0BB
:1034B000100B01E16BD11ED02EDBE3DB70DA91EC57
:1034C0001EF006E1CBD9020EEF6E06EC28F02BD0F1
:1034D000C5D9030EEF6E100EB86FEDDB0001F85189
:1034E000F91168E1C1D06CEC1EF0000920E1D9DBD4
:1034F000020B03E10701040E18D00DDBDCDB0A0E22
:10350000E66EE66AF4C0E6FFF5C0E6FFA7D9DDD9AE
:103510001250B3D9F7D9A2D9D4DAA0D9020EEF6EDE
:1035200019DB36DB3CDA0701120EB86FDAD0A9DB03
:10353000EECFAEF7EECFAFF7EECFB0F7EFCFB1F7FC
:1035400009DBEECFB2F7EECFB3F7EECFB4F7EFCFA4
:10355000B5F793D9040E7ED922DA0001F85107019C
:10356000A6270001F9510701A723000EA823A923CC
:10357000F1DA49DB040E6ED9EE50AE1901E0A4D0A9
:10358000EE50AF1901E0A0D0EE50B01901E09CD090
:10359000EE50B11901E098D001E096D09DDB020811
:1035A0000BE1BFDB61E008DB030EEF6E0001F851B9
:1035B000F9115AE06ADB95D0FFDAEF50030857E1C2
:1035C000B0DB29E05AD9080E45D9EECF10F0EECF86
:1035D00011F067DABFDA1050EE181DE11150EE1845
:1035E0001AE11250EE1817E11350EE1814E113E12E
:1035F00035D944DB020B0FE131D935D905E1115042
:1036000003E1125001E1135006E028D9ACD926D9C4
:10361000F6DA84DBEF8277DA010B09E00701110E9D
:10362000B86F98DAB5DA7DD919D9090EEF6E0001B5
:10363000F851F91119E012D968DB04E126DB070122
:10364000B8894FD087DAB2C7EEFFB3C7EEFFB4C771
:10365000EEFFB5C7EEFF15DBAEC7EEFFAFC7EEFF5F
:10366000B0C7EEFFB1C7EEFF06EC28F03AD034DB6E
:10367000090804E116DB100B34E020D02DDB040830
:103680000FE10FDB010B06E0C8DA4BDB17E1E6D8F0
:10369000060E04D046DB25E0E1D8050EEF6E21D002
:1036A0001BDB050805E1FDDA010B1BE0B6DA06D0ED
:1036B00013DB060816E1F5DA100B13E0B6C7F1F0DC
:1036C000B7C7F2F04ADE0DD006EC28F00701100E65
:1036D000B86FAEC7A6F7AFC7A7F7B0C7A8F7B1C70F
:1036E000A9F70701B85152E0B9D8C8DA020B2FE1A7
:1036F000B5D8B9D805E1115003E1125001E11350DA
:1037000026E0ACD8100E77DA22E0DBDA1050EE5E5D
:103710001150EE5A1250EE5A1350EE5A9FD89FDABB
:103720009DD80F0EEB500001E86FB8C710F07BDAA0
:10373000108610C0E7F053DA0DDA0CD98FD853DABF
:103740008DD855DA8BD8FAD8BCDA42EF1DF064D99F
:10375000B8C7E7F0A6C7E3F0A7C7E4F0A8C7E5F04D
:10376000A9C7E6F0AAC7DFF0ABC7E0F0ACC7E1F04D
:10377000ADC7E2F082D841D980D8020E6BD842D9C9
:10378000F4C0D9F0F5C0DAF0BAEC17F0120000017D
:10379000FA51240DF3CF10F0F4CF11F0000E1026E3
:1037A0000A0E112210C0F3FF11C0F4FF1200000135
:1037B000FB51240DF3CF8DF7F4CF8EF7000E0701E8
:1037C0008D270A0E8E230C0E04019B6F9C6BF1EC6F
:1037D0004BF0FCEC26F0E840E8403F0B3C0B0701C7
:1037E0008C6F0001FC51B15D106EB251FD55116E30
:1037F0008DC7E9FF8EC7EAFF120E10C0EBFF130E54
:1038000011C0EBFF07018C510001FC2504019B6FE7
:10381000000E0001FD2104019C6FF1EF4BF000014F
:10382000FE51240DF3CF00F7F4CF01F7000E07018E
:1038300000270A0E012300C7E9FF01C7EAFF62DA89
:103840000001EE50B15D106EEE50B25910C0F3FFA2
:10385000F46E1200E926000EEA221200B6C7E9FF54
:10386000B7C7EAFF12000F0EEB50106E78EF1EF094
:1038700075C7E9FF76C7EAFF1200F6C0E9FFF7C097
:10388000EAFF1200EFC0E9FFF0C0EAFF12001E0ECF
:10389000EB50106EC8D9D880030E1054000E26EFDE
:1038A0001EF0240DF3CFE9FFF4CFEAFF000EE92666
:1038B0000A0EEA2212006DC7E9FF6EC7EAFF120086
:1038C000F1C0E9FFF2C0EAFF1200EE52E9CF10F0BA
:1038D000EACF11F0E9CFE6FFEACFE6FFC0EC55F002
:1038E000126E060EE15E1200EECFE3F0EECFE4F0D2
:1038F000EECFE5F0EFCFE6F0120076C7E9FF77C72D
:10390000EAFF1200EECF10F0EFCF11F012006CC7FB
:10391000E9FF6DC7EAFF120000C7E9FF01C7EAFF30
:103920001200EF2AEECFA6F7EF22EECFA7F7EF2295
:10393000EECFA8F7EF22EFCFA9F71200EE52E9CFB2
:10394000D9F0EACFDAF0BAEF17F001C7E9FF02C702
:10395000EAFF1200EECFDFF0EECFE0F0EECFE1F0C5
:10396000EFCFE2F012000F0EEB500301BB6FFBEF45
:1039700027F001C7E9FF02C7EAFF12006CC7E9FFA1
:103980006DC7EAFF120074C7E9FF75C7EAFF1200AE
:10399000101649D910501110121013101200EECF4A
:1039A000A6F7EECFA7F7EECFA8F7EFCFA9F7120053
:1039B00011C0EEFF12C0EEFF13C0EEFF120000C7F1
:1039C000E9FF01C7EAFF120087C7E9FF88C7EAFFDE
:1039D00012001850145C106E19501558116E1A50C0
:1039E0001658126E1B501758136E12000301CD6F3C
:1039F000CE6BE8C0CCF321EF2AF0EECFDDF0EDCFB7
:103A0000DEF01200EECFDBF0EDCFDCF0120087C766
:103A1000E9FF88C7EAFF12000001E96BEA6B0001C9
:103A2000E8691200126A136ACA0E105C030E11587C
:103A3000000E1258000E135812001F0EF9C2EBFFB1
:103A4000200EFAC2EBFF12000F0EEB500301CC6FF9
:103A500021EF2AF007017851F00BE842E842E842F2
:103A6000E842040DF3501200240DF3CF00F7F4CF19
:103A700001F7000E00270A0E01231200E552E7505D
:103A8000EF6E12001050EE261150EE221250EE2270
:103A90001350EE221200EDD8280E0301CD6FCE6B2D
:103AA0001200EECF12F0EFCF13F01200E8C010F0CA
:103AB00078EF1EF00301010EAB6F17EC26F0000942
:103AC00012000D0E10C0EBFF0E0E11C0EBFF120026
:103AD000140E10C0EBFF150E11C0EBFF12002C0EE0
:103AE000EE6E010EED6E1200EE6AEE6AEE6AEE6A9E
:103AF0001200EE2AEE22EE22EE221200EBC0E9FFC7
:103B0000ECC0EAFF1200B9DE0D0EA4DEEF50120089
:103B1000230E2AEF1CF0F8C014F0F9C015F0166A55
:103B2000176AABDE040E96DEEE501424106EEE50D3
:103B30001520116EEE501620126EEE501720136EE7
:103B4000102A000E1122122213229BD810C0EEFF61
:103B5000D8EF1CF083DE58EF1EF07CDE6FEF1EF016
:103B600079DEEECF3BF3EECF3CF3EECF3DF3EFCF7C
:103B70003EF315EC36F004C010F005C011F006C09D
:103B800012F007C013F042EF1CF064DE82EF1CF06D
:103B9000EFCFAAF7EE2AEFCFABF7EE22EFCFACF7DD
:103BA000EE22EFCFADF7EF2241EF1EF0010E52DE15
:103BB00007C7EFFF42EF1CF064D8A6C7EEFFA7C708
:103BC000EEFFA8C7EEFFA9C7EEFF2EEF1CF042DE06
:103BD000EFCF07F742EF1CF08FD842EF1CF01A0E20
:103BE00039DE74EF1CF00D0E35DEFDEF1CF00B0E10
:103BF00031DE02EF1DF02EDEEE50ED1012000F0E42
:103C000029DEEF681200EECFAAF7EECFABF7EECFCA
:103C1000ACF7EFCFADF73DEF1CF00701100EB86F1A
:103C200030D891EF1CF0116A126A136A120043DE59
:103C30003FD85FDF5BEF1CF00DDE04C0EEFFB8DEA7
:103C400042EF1CF0210E06DE6FEF1DF01154000E46
:103C50001254000E135412000BDE47EF1CF0100E2E
:103C6000F9DDEECFE9F0EDCFEAF01200060E2AEF13
:103C70001CF0100EEB6A110EEB6A120049DFEF50D8
:103C80001200ECDD1A0E2AEF1CF048D8EF86E6DDB4
:103C9000120EF8C0EBFF130EF9C0EBFF3FD8EF8414
:103CA000120006EC28F083EF1DF063DE88EF1DF0B4
:103CB000160E2AEF1CF0E1DD0E0E67DFCFDD68EF98
:103CC0001DF0CCDD100E61DF126A136AAAEF1DF041
:103CD0001EDE100E2AEF1CF0C1DDEF501200010EA7
:103CE000B9DDEF50E66E42EF1CF02FDE88EF1DF0DD
:103CF0009ADFE86810181200ADDD3EEF1DF0AADD76
:103D0000D6EF1DF0120E2AEF1CF0B8DF080B1200E0
:103D1000FFDEEF961200CCDFAAEF1CF09FDD88EFEC
:083D20001DF0F1DE100B120092
:083D2800F9C2A4FBFAC2A5FBDD
:103D30000701036B060E035D2DE2750EEAEC24F01D
:103D4000116E106A10C0E6FFE66E740EEAEC24F005
:103D5000E552E7CF11F0E552E7CF10F00001101067
:103D6000B36F11C0B4F037EC12F0E66E07013BEC14
:103D700024F0E552E750EF6E3BEC24F0020E08EC25
:103D800024F0EF6A3BEC24F0090E08EC24F0EF6A13
:103D9000032BD0D712000701D56B060ED55D06E2C6
:103DA000D5C7ABFB96D80701D52BF7D71200A6CB0A
:103DB00000F7A7CB01F7070100C7E9FF01C7EAFF3A
:103DC000002B000E0123EF502E0807E000C7E9FF8B
:103DD00001C7EAFFEF50EFE10A0C026B0251106ECF
:103DE000116A100E105C000E115821E28FEC24F0C5
:103DF00002C716F0176A186A020ED89016361736E0
:103E00001836E806FAE114EC24F000C7E6FF01C713
:103E1000E6FF25EC56F0196E050EE15E195000091B
:103E200003E10701025112000701022BD7D70A0C48
:103E300063EC24F004E0200E0701005DF9E00701C7
:103E4000016B2B0E0701005D02E1200E006F2F0EAB
:103E5000005D20E05C0E005D1DE0200E005D1DE0B9
:103E60003F0E005D1AE00D0E005D17E00A0E005DCA
:103E700014E00C0E015D0EE2610E005D05E30051E1
:103E80007A0802E3200E005F0151012B96EC24F02A
:103E900000C7EFFF63EC24F0D4E10701015196EC79
:103EA00024F0EF6A070101510EE1C30EE66EB70E72
:103EB000E66E000EE66EA9CBE6FFAACBE6FF3BEC72
:103EC00056F0050EE15E3F0E0701005D01E1010CB9
:103ED000000C0B01AB510A0DF3CFC5F7F4CFC6F7B9
:103EE000680E0701C5270B0EC623010EC36F07011D
:103EF000C35101E143D2C36BCC6B03EC24F09DECC6
:103F000024F00DE119EC25F0020B02E014EC25F091
:103F1000BBEC24F0EF94BFEC24F0EF6A120003EC4A
:103F200024F0020EEB50080AE2E00F0A01E112D27F
:103F3000010A01E1E2D1030A01E1DFD1010AD7E080
:103F4000070A01E103D2010A01E1B7D1030A01E145
:103F500072D1010ACCE103EC24F0AAEC24F0C7E012
:103F60000701010EC36FF9C2A4FBFAC2A5FBBBECAB
:103F700024F0EF6AF6EC24F00B01B16F5CDA070174
:103F8000C26F0B01B50EA96F070EAA6FF6EC24F0F5
:103F90000B01A86F4DDF0701CC91E8B0CC81F6ECA6
:103FA00024F00001FE6F0FEC1CF0F3CFCAF7F4CF42
:103FB000CBF70B01B50EC16F070EC26FABCBC0FBC9
:103FC00097DB0B01B50EA66F070EA76FF0DEE66E4E
:103FD000B9EC24F0E552E750EF6E0DEC25F0060E3B
:103FE000101805E1115003E1125001E113502CE0CB
:103FF000B9EC24F0EFCF14F0156A166A176A010EB7
:10400000141805E1155003E1165001E1175002E0C4
:10401000000E01D0010E000E000916E1B9EC24F0EB
:10402000EFCF18F0196A1A6A1B6A040E181805E116
:10403000195003E11A5001E11B5002E0000E01D0BB
:10404000010E000E000904E0BBEC24F0EF8003D069
:10405000BBEC24F0EF90E5DB020B25E10DEC25F045
:10406000060E101809E1115007E1125005E1135036
:1040700003E1D7DB100B17E1580E0701B55D03E133
:10408000D0DB010B10E119EC25F0010B03E0C9DBDB
:10409000080B09E1C6DB040B0DE00701C2510AE180
:1040A000CC51010B07E019EC25F0040B03E1FDEC0A
:1040B00024F03CD00701C25101E0B7D0BBEC24F0A2
:1040C000CC93EF50040B01E0CC83ABDB200B03E17E
:1040D000BBEC24F0EF840701CCA115D0CAC7FCF0DB
:1040E000CBC7FDF0F6EC24F00001FB6FD7EC1BF022
:1040F0000401B50EE46F070EE56FC5C7E2F4C6C74D
:10410000E3F4A1EC57F0BBEC24F00701CC51020B17
:1041100002E0EF8401D0EF94FDEC24F019EC25F0DF
:10412000100B0CE019EC25F0040B08E10BEC25F06A
:10413000020EEF6E68DB6CDB060E0AD1BFEC24F0DA
:10414000050EEF6EC5EC24F000EC25F0060ED7DB73
:1041500046E30DEC25F0D880040ED9DB40E3B50E24
:10416000E66E070EE66E54EC56F0E552E552F3CFDC
:10417000C4F70DEC25F0D880030EC9DB02E3030E73
:1041800001D0020E0701C45F0DEC25F00B0E1026C6
:10419000000E112212221322ECDB10C0EFFFBFDB56
:1041A000E8DBEFCF16F0176A186A020ED8901636C1
:1041B00017361836E806FAE137DB0701C4511A6AE8
:1041C000B50F196E070E1A2219C0E6FF1AC0E6FFD6
:1041D0003BEC56F01B6E050EE15E1B50D6DB00EC8F
:1041E00025F0E86810180AE1115008E1125006E1C4
:1041F000135004E10BEC25F0EF6A0FD000EC25F032
:10420000FE0E10180DE111500BE1125009E1135090
:1042100007E10BEC25F0010EEF6EB1DB050E98D037
:10422000AADBEF82ACDB010E93D0C20501E05FD6C2
:10423000A6DB030E8DD0E7DB01E159D60701010EA5
:10424000C36F0B014C0EBD6FB70EBE6F000E36DB99
:104250008CDB0B015C0EBD6FB70EBE6F000E2EDB4C
:1042600088DB7FDBC50EE9260B0EEA22EECFBDFB15
:10427000EECFBEFBEFCFBFFBABCBBCFB0FDA75DBEA
:10428000CCDB0B0E3CDB07E30B016B0EBD6FB70EF7
:10429000BE6F000E13DBCDDB010B07E10B01B40E8B
:1042A000BD6F8E0EBE6F000E09DB5FDBACDA030E56
:1042B000AFDAEF6A64DB020E4BD0A5DA4BDB01E02C
:1042C0009CDB59DB0701CC93EF50040B01E0CC835E
:1042D000A8DA200B02E14FDBEF84ABCBB2FBEED8C8
:1042E000000904E0A1DB4BDB070EEF6E44DB0701A6
:1042F000CC51020B41E0EF84FAD585DB01E1F7D523
:104300008ADB2FDBF50EE9260B0EEA22EECFC7F78C
:10431000EECFC8F7EFCFC9F70701C7C7F6FFC72B26
:10432000C8C7F7FF000EC823C9C7F8FFC923080094
:10433000F5CFC4F7F55005E0C4C7BEF064DAAEDAD5
:10434000EBD754DB0001BB6F4DEC13F018DB070E0D
:10435000EF6ECDD558DAF1DA0AE055DB08E046DB3E
:104360000001BA6F0AEC13F00ADB080EEF6E4BDAAD
:10437000090EE926000EEA22EF94B9D51200AFCB60
:10438000E9FFB0CBEAFFEF0407014A6F496BEF6A20
:104390004B6B4A510B01EA6AAD25E96EAE51EA2238
:1043A000EF6A07014B5141E10001480ED06F070E43
:1043B000D16FACCBCFF097EC15F0000936E03D0E95
:1043C0000701485D0BE1486B4A51495D1EE24929EE
:1043D000AFCBE9FFB0CBEAFFEF6E17D0260E485DFA
:1043E00002E1020E0AD0200E485D06E00D0E485D87
:1043F00003E00A0E485D04E1010E4B6F486B05D0E7
:104400002B0E485D02E1200E486F4A51495D06E2DD
:10441000ADCBE9FFAECBEAFF48C7EFFF0B01AD2BF9
:10442000000EAE230701492BBCD707014B5101E118
:10443000000C4B0512000701056B0001060ED06F42
:10444000070ED16FB1CBCFF097EC15F0000916E055
:10445000200E0701065D12E00551106E116A040E70
:10446000105C000E1158E9E20551052BEA6A000FB5
:10447000E96E070EEA2206C7EFFFDFD707010551F5
:10448000EA6A000FE96E070EEA22EF6A470E005D46
:1044900007E1450E015D04E1540E025D01E1000CEF
:1044A000500E005D0AE14F0E015D07E1530E025D03
:1044B00004E1540E035D01E1010C020C0B01B25149
:1044C0000A0DF3CF6EF7F4CF6FF7680E07016E2772
:1044D0000B0E6F23A1D9DBD901E1C5D007016C6BAD
:1044E0009BD9030EEB5004081AE096D9DCD9400E94
:1044F000FAD90EE191D9010EEB500201806F5BEC0D
:104500003FF007016D6F88D9CED9200EECD907E0B6
:1045100083D9EF500001BB6F4DEC13F0010C7CD937
:10452000090E76D9EF50010B01E196D075D9030E33
:10453000EB50040A65E0070A35E0010A1CE0030AB3
:104540000CE0010A01E085D0250E6D5D03E12DDA56
:10455000010E26D0010E6C6F7CD0250E6D5D03E13F
:10456000010E6C6F74D00FDA030E52D96DC7EFFFD6
:104570001CDA020E15D0610E6D5D02E3270E04D029
:10458000410E6D5D02E3070E6D5F300E6D5D100D27
:10459000F350E66E45DAE552E750EF6E06DA030EA9
:1045A000EF6E57D0610E6D5D02E3270E04D0410E11
:1045B0006D5D02E3070E6D5F300E6D5D106E30DADB
:1045C0001050EF12F2D9040EEF6E26D921D9EE6AFF
:1045D000ED6A0B01B56BB66B23DAEFCFB3FBD3D922
:1045E000030E16D9EFCFB4FB6D0EB76F070EB86F81
:1045F0006EC7C3FB6FC7C4FBFDD80B01B96F29D0D1
:10460000C2D9EECFB5FBEDCFB6FB0301B30EDC6F25
:104610000B0EDD6FC9EC0DF0B6D9B5CBEEFFB6CB06
:10462000EDFF0701010E6C6FB5CB10F0B6CB11F0AA
:10463000126A136AE86810180CE1E868111809E1B9
:10464000125007E1135005E16D5101E16C6BADD9DA
:10465000EF6A07016C5104E06DC7BEF0DDD81ED9CA
:10466000D7EC45F037D7D8D8010EEB5002017F6F59
:104670002DEC3FF0000C0B01BB510A0DF3CF6CF792
:10468000F4CF6DF7680E07016C270B0E6D23000148
:104690000D0EA5D900010A0EEFEF24F00B01BC515D
:1046A0000A0DF3CF6CF7F4CF6DF7680E07016C2796
:1046B0000B0E6D23BDCBF6FFBECBF7FFBFCBF8FFD4
:1046C0000800F55014E00B01BDCBF6FFBD2BBECBAF
:1046D000F7FF000EBE23BFCBF8FFBF230800F5CFC6
:1046E000BEF06CC7E9FF6DC7EAFFD8D8E3D7120068
:1046F0000B01C0510A0DF3CF00F7F4CF01F7680E9C
:10470000070100270B0E0123040E836F00010A0E20
:10471000A5D805E1115003E1125001E1135006E064
:104720000701835183070009F1E1120000010D0E1A
:10473000CE6F0001800ECD6F0001020ECB6F070E11
:10474000CC6F37D9F3CF85F7F4CF86F7F4CF10F0DD
:1047500050D9F45011101210131015E10701040E76
:10476000836F00010D0E7AD805E1115003E112505C
:1047700001E1135005E00701835183070009F1E1CE
:104780000701200E866F86C710F033D9200E10184F
:1047900005E1115003E1125001E1135001E0120054
:1047A0000701850501E112000001830ED06F070E9D
:1047B000D16F00C7E9FF01C7EAFFEF500001CF6FDB
:1047C00097EC15F007018505EA6A020FE96E070EFE
:1047D000EA22EF6AC1CBC7F4C2CBC8F40401020ECF
:1047E000C56F070EC66F00C7C3F401C7C4F4B7ECAA
:1047F00046F09CD7E7D8040B05E0E4D8080B01E0AD
:10480000020C010C000CC5C7E9FFC6C7EAFF120085
:10481000E926000EEA2212006EC7E9FF6FC7EAFF21
:104820001200720EEAEF24F013501624F36E1450A7
:104830001720F46E15501820F86EF4CFF7FFF3CF61
:10484000F6FFF6CF10F0F7CF11F0F8CF12F010C04E
:10485000E6FF11C0E6FF12C0E6FF1200CE6F0001B6
:10486000CD690001CB6BCC6BA4D8F4CF10F0C1D8CC
:10487000200EF418120003510A0DC8D8680EE9265C
:104880000B0EEA221200EFCF10F0F9EF24F0EF50F8
:104890000001BC6FA3EC13F000091200EF500001FF
:1048A000BD6FCEEF13F0010EEB50080DAFD8480EE0
:1048B000E926020EEA22EFCF10F01200BF6FABCB59
:1048C000BCFB4EEF23F00001000ED06F070ED16F3E
:1048D000A8CBCFF097EC15F000091200010EEB50B9
:1048E000106EF9EF24F0101684D810501110121029
:1048F00013101200EF500001C46FBBEF14F0105CF6
:10490000000E1158000E1258000E135812001054C9
:10491000000E1154000E1254000E135412000C0E0F
:10492000136EB70E146E000E156E12000B01EA6ABC
:10493000A925E96EAA51EA221200EF500001B96FD1
:1049400001EC13F000091200010EEB5002017E6F22
:1049500025EF3FF0EF500001D26FD6EC15F00009C3
:104960001200EF50030D06EF25F0ABCBBBFB3BEF86
:1049700023F051D861D047DF090E08EF24F043DF60
:10498000020E08EF24F048DF57D002017D6B0201D0
:10499000B50E7B6F070E7C6F71EC3EF0E66E33DF79
:1049A000EE52E552E750EF6E120036DF030E08EFCD
:1049B00024F000C7E9FF01C7EAFFEF500001CA6F0A
:1049C00028EF15F0C3CBE9FFC4CBEAFF090E20DFC7
:1049D000EF50120003012A6F2B6B42EF43F0BE6FC2
:1049E0006CC7E9FF6DC7EAFF4EEF24F00CDFEF5014
:1049F0001200116A126A136A120005DF7AEF24F0BE
:104A000002DF6EEF24F0FFDE47EF24F0F3CFE9FF83
:104A1000F4CFEAFF1200F7DE0FD0ABDF43EF24F054
:104A2000B2DF020E08EF24F0A6DFEF92ECDEA4EF77
:0E4A300024F0A1DFEF501200040E08EF24F076
:024A3E00966A76
:104A4000868898880301A56BA66BA76BA86BA96BDA
:104A5000AA6B0701006B00C710F04DEC2AF01EE2B4
:104A600000C710F0CDEC2AF0020ED89010361136A7
:104A700012361336E806F9E1400E1026000E112218
:104A8000122213220701005138EC2AF010C0EFFF68
:104A90000051ADEC2AF0EF80002BDDD7236A030133
:104AA000A369CBEC29F068EC2AF003011F0E52EC4D
:104AB0002AF00301C66F03011F0E9FEC2AF068EC79
:104AC0002AF00301210E45EC2AF068EC2AF00301DC
:104AD000080EC66F03010E0EA9EC2AF00A0EA9EC0F
:104AE0002AF00B0E4AEC2AF0040EC66F03010C0EDE
:104AF0004AEC2AF0020EC66F03010D0E9FEC2AF05D
:104B0000BBEC2AF09BEC2AF0010E4AEC2AF0600E76
:104B1000C66F0301020E4AEC2AF09BEC2AF0030E4A
:104B20004AEC2AF0C6690301070EA9EC2AF00F0E21
:104B30004AEC2AF0610E45EC2AF004C3C6F30301E7
:104B4000010E9FEC2AF005C3C6F30301020E9FEC91
:104B50002AF006C3C6F30301030E9FEC2AF007C335
:104B6000C6F30301040E9FEC2AF008C3C6F3030149
:104B7000050E9FEC2AF009C3C6F30301060E9FEC55
:104B80002AF00701006B080E005D13E20301C669FD
:104B900000C710F0CDEC2AF0080E1026000E1122EE
:104BA0001222132210C0C5F3DAEC29F00701002B02
:104BB000EAD703019BEC2AF0070E9FEC2AF04C0E7B
:104BC000206E0301220E45EC2AF00301C66B03019F
:104BD0000D0E4AEC2AF0E00E45EC2AF00301C00E5F
:104BE000C66F0301010EA9EC2AF0040EA9EC2AF00D
:104BF000010E4AEC2AF0200E45EF2AF003010D0EBB
:104C0000C8EC2AF00301A5271150A62303010E0EBC
:104C1000C8EC2AF00301A7271150A82303010F0EA7
:104C2000C8EC2AF00301A9271150AA23120003019E
:104C3000AB5105E06DEC2AF001E0000C010CA35132
:104C4000235C05E16DEC2AF001E0000C010C07018A
:104C5000010E926F92C710F04DEC2AF007E29251CC
:104C6000D6EC2AF001E0010C922BF4D7000C0301E2
:104C7000AC5108E06DEC2AF002E1106A01D0106836
:104C8000105012000701010E926F92C710F04DEC08
:104C90002AF010E29251D6EC2AF00AE09251ADECE3
:104CA0002AF0EF909251ADEC2AF0EF92925112005F
:104CB000922BEBD7FF0C8BEC2AF086A8FED772EC78
:104CC0002AF086A8FED792EC2AF086A8FED78D8C13
:104CD000670E8D6E400E836E8D9C86A8FED78D8CE0
:104CE000700E8D6EADC383FF8D9C86A8FED78D8C14
:104CF000212A000E222212000301B051B11101E15C
:104D00001200010EB015106E116AB0511024070187
:104D1000CF6F0301B15111200701D06F956A670E63
:104D20008D6E400E836E8D9C86A8FED78D8C6A0E8C
:104D30008D6ECFC783FF8D9C86A8FED78D8C6B0EA2
:104D40008D6ED0C783FF8D9C86A8FED792EC2AF08B
:104D500086A8FED78D8C0301B0512126B1512222A5
:104D6000700E8D6EB0EC2AF086A8FED78D8CB0C385
:104D7000CDF7B1C3CEF70701010ECD5F000ECE5BBC
:104D80000701CDC710F0CEC711F0CD07000ECE5BE6
:104D90001050111030E0080ECD5D000ECE5926E304
:104DA00071DB86A8FED78D8C6DDB86A8FED78D8C37
:104DB00069DB86A8FED78D8C65DB86A8FED78D8C37
:104DC00061DB86A8FED78D8C5DDB86A8FED78D8C37
:104DD00059DB86A8FED78D8C55DB86A8FED78D8C37
:104DE000080E0701CD5F000ECE5BD5D74BDB86A842
:104DF000FED78D8CC5D712008EDB86A8FED772DB5E
:104E000086A8FED78D8CFF0E215C1DE12250106E0E
:104E1000C4DB5F0E221817E1115015E1125013E1A7
:104E2000135011E1070193695F0E68DB61DB86A80F
:104E3000FED78D8C0301100E35DB0701926F936B4B
:104E40004C0E5CDB10D054DB86A8FED78D8C9568A9
:104E5000700E8D6E8D9A86A8FED783CF92F78D8ABD
:104E6000212A000E2222070192511200B4C392F7A8
:104E7000B5C393F70301B451B51103E1F36AF46AC2
:104E80001200956A6A0E8D6E92C783FF8D9C86A86C
:104E9000FED78D8C6B0E8D6E93C783FF8D9C86A87D
:104EA000FED78D8C25DB86A8FED78D8C070192510D
:104EB00021269351FADA02E3140E225E9568700EF1
:104EC0008D6E070192C710F093C711F09207000E84
:104ED000935B105011100FE08D9A86A8FED7030146
:104EE000B2C3E9FFB3C3EAFFB22B000EB32383CFF3
:104EF000EFFF8D8AE6D7B4C3F3FFB5C3F4FF12000A
:104F0000B8C38CF707018D6B0301B85103E1F36A55
:104F1000F46A1200956A6A0E8D6EB8C383FF8D9C89
:104F200086A8FED7DFDA86A8FED78D8CE1DA86A8C0
:104F3000FED78D8C9568700E8D6E07018C512DE01B
:104F40008C078D9A86A8FED783CF8EF78D8A0301B2
:104F5000B651B71109E0B6C3E9FFB7C3EAFFB62BF4
:104F6000000EB7238EC7EFFFB95107018E5DE5E153
:104F7000200E8D6F956A600E8D6E200E836E8D9C57
:104F800086A8FED78D8C6A0E8D6E836A8D9C86A84E
:104F9000FED7A8DA86A8FED78D8C07018C510301B5
:104FA000B85D07018C6FE850116AE8502126115056
:104FB0007CDA02E3140E225E8DC710F0EEDA200ECA
:104FC00010180BE1115009E1125007E1135005E1EF
:104FD00021C0C8F322C0C9F307DA126A07018C5155
:104FE00000011210F36E8DC7F4FF12000301BA51D5
:104FF000B4DAEF901200BBC310F04FDA06E20301FF
:10500000BB51ABDAEF80BBC323F0120020C097F78F
:105010000701010E966FE8CFC8F320C0C9F3E4D9A9
:10502000EBDE0701956FE8CFC6F30301030E81D2D3
:10503000AADA0701006F0301200E27DA20500701CA
:10504000005D1CE2600E146E156A166A176A205025
:10505000186E196A1A6A1B6A20502EDA00C71CF0F3
:105060001D6A1E6A1F6A1C5010261D5011221E50F8
:1050700012221F50132210C001F703D02050005DF0
:10508000016F140E146E156A166A176A01C718F0BC
:10509000196A1A6A1B6A18500FDA10C001F710C09B
:1050A00003F7026B02C7F3FF10C0F4FF1200030105
:1050B000E00E77DA0701006F0301200EE6D9070141
:1050C0000051040B01E0000C010CBEC3E9FFBFC39B
:1050D000EAFFEF6858DA0701126F0301200E61DA68
:1050E0000701136F67DA100B42E0F7D90701166F5B
:1050F0000301210ECAD90B01020EFF6FA9EC5CF06F
:105100000301C66B03010A0E24DA0B0E18DA07013D
:10511000165108E04FDA0A0B02E0000E01D0010E32
:105120000701166F0301020EC66F03010D0EB2D9FF
:10513000220EABD912C720F069DF0301FCD9030EA0
:10514000A9D9620EA2D90301F6D9070EA3D9220E5E
:105150009CD90301C6690301070EFBD90D0EEFD9D7
:105160000701165103E00301260E8FD9000C070139
:105170001351125D01E192D013C715F7146B14C7D8
:10518000C8F313C7C9F330D9120E0301B46FB56B5E
:105190000301000EB26F070EB36F68DE0701005106
:1051A000010B01E178D002C710F003C711F0126AB9
:1051B000136A400E105CC6D96EE302C714F003C731
:1051C00015F0166A176AD880EE0E1454050E1554A1
:1051D000000E1654000E17545EE301C718F0196A4A
:1051E0001A6A1B6A600E185C000E1958000E1A58D5
:1051F000000E1B5850E201C71CF01D6A1E6A1F6A90
:105200004C0E1C5C000E1D58000E1E58000E1F5840
:1052100042E310C739F311C73AF310EC36F0F3CF7D
:1052200010F7F4CF11F7060EE66EE66A0A0EE66E88
:10523000070EE66EBCC3E9FFBDC3EAFFBCC310F0B6
:10524000BDC311F0BCC3E6FFBDC3E6FFC0EC55F023
:10525000126E060EE15E1250080E0701115D18E194
:1052600010C710F052D90EE010C714F0156A166A74
:10527000176A060E14180CE115500AE1165008E1E1
:10528000175006E1BEC3E9FFBFC3EAFF10C7EFFF37
:1052900013C720F0010C12C720F0B8DE000C030188
:1052A0000A0EC66F0301070E4AD92350E1D8EFCF8B
:1052B000D2F70701D16BD1C7C8F3D2C7C9F394D8CD
:1052C000060E0301B06FB16BC0C3AEF3C1C3AFF341
:1052D00013DD04C3ADF3EFDC05C3ADF3ECDC06C3B3
:1052E000ADF3E9DC07C3ADF3E6DC08C3ADF3E3DC03
:1052F00009C3ADF3E0DCC2C310F007D903E1070135
:10530000D36B03D00701060ED36F0301080EAD6FF8
:10531000D2DCD3C7ADF3CFDC0E0E0301C327000EE2
:10532000C423C3C310F0C4C311F0126A136A3C0E45
:10533000105C08D903E23C0EC36FC46BC3C3D1F742
:10534000C4C3D2F7C3C3C6F30301050EF8D8D2C74E
:10535000C6F30301060EEDD00ED9240E96D823C055
:10536000A3F32350FAD8EF802350F7D8EF82070138
:10537000926B92C710F091D80DE2925117D907E0C5
:1053800092510301A35D03E092C723F012000701CD
:10539000922BEFD712009568600E8D6E8D8C8D8AE2
:1053A0008D8E966A0B01010EFE6F9CEC5CF090D81E
:1053B0008D9E1200600E0301C5118D6EC6C383FF62
:1053C000956A8D9C86A8FED78D8C12009568600E1C
:1053D0000301C7118D6E8D9A86A8FED783CF98F7EB
:1053E0008D8A070198511200C8C321F0C9C322F069
:1053F000C8C3C6F30301080EA2D8C9C3C6F303018C
:10540000090E97D00301090E4DD80701016F030162
:10541000080E48D8F36E01C7F4FF120020C093F7BE
:105420000701120E926F0301CA510701922703016F
:10543000CB510701932392C7C8F393C7C9F3F4EF85
:1054400029F0CCC323F0235013D8EFCF93F70701F3
:105450000E0E926F0301CD51070192270301CE5129
:105460000701932392C7C8F393C7C9F3F4EF29F058
:10547000E96EEA6AD890E936EA369D0EE926030E0F
:10548000EA2212000301B0EF2AF0C66F0301C56BD8
:10549000DAEF29F054D8030112007FD8030E105C14
:1054A000A2EF2AF0C76FE6EF29F02222225075D82A
:1054B000600E225CA2EF2AF0145C106E1950155891
:1054C000116E1A501658126E1B501758136E120098
:1054D0000B01050EFF6FA9EF5CF00301C76B76DFD0
:1054E000040B12008D8C6B0E8D6E836A8D9C1200E6
:1054F000600E8D6E0A0E836E8D9C1200946F93C7A2
:10550000C8F3E8CFC9F3F4EF29F047D810501110D1
:10551000121013101200956A6A0E8D6E010E836EC2
:105520008D9C12008D8C600E8D6E120E836E8D9C84
:1055300012009FEF2AF04C0EC66F03011200C56FD8
:10554000DAEF29F0000E1158000E1258000E135811
:105550001200A0DFC66B030112008ADFEE521200B8
:10556000AEC3E9FFAFC3EAFFAE2B000EAF23EF508F
:10557000836E8D9C120023507BDFEFCFC6F30301B7
:10558000040E4AEF2AF00301600E7FDFDAEF2AF003
:1055900089DF106E116AE8501200116A126A136AEC
:1055A000120073DF0301030E52EF2AF0D6DFEF5033
:0C55B000010B12000301070E52EF2AF05D
:0455BC000701006B78
:1055C000080E005D06E200C7A7F151D80701002BC5
:1055D000F7D712000701000E5B6F010E5C6F5A6B6C
:1055E000080E5A5D43E25EDB0C0E49DB4CDB126AAF
:1055F000136A105011101210131032E153DB0C0E0D
:10560000A1C1EBFF0D0EA2C1EBFF0101A351A4113B
:1056100011E00A0EE66EE66AA3C1E6FFA4C1E6FF4A
:1056200041DB5BC710F05CC711F05BC7E6FF5CC7EE
:10563000E6FF63DB37DB0A0EA5C1EBFF0B0EA6C14D
:10564000EBFF30DB0E0EEB6A0F0EEB6A2BDB100E5E
:10565000EB6A110EEB6A5AC7A0F107015A5112000A
:10566000140E5B27000E5C235A2BBAD7FF0C0101E6
:10567000A751FBDA0C0E03DBEE6AED6AA751F5DAEF
:10568000060EFDDAEE6AEE6AEE6AEE6AA7515DDB9F
:10569000EF901200080E0101A85D07E2A8C1A0F179
:1056A0000301010EAB6F17EF26F0000C0101A051B2
:1056B000140DF3CF59F7F4CF5AF7000E070159270D
:1056C000010E5A234ADBEE50ED1016E11DDBEFDA36
:1056D00048DBEDDA120EEB50106EF3DA07E11150F1
:1056E00005E1125003E1135001E1000C1C0E03010F
:1056F000CD6FCE6BDCDAFBDAA9C1ADF35BEC26F043
:105700002CDBEE2AEF2229DBBEDAE6DA01E374D8DD
:10571000010C0101A051140DF3CF41F7F4CF42F772
:10572000000E07014127010E422313DBEE50ED105E
:1057300018E1EADAADDA15DBABDA120EEB50106ED7
:10574000C0DA09E1115007E1125005E1135003E1FD
:10575000F36AF46A12001C0E0301CD6FCE6B98DA67
:10576000C6DAF7DA0101AC51EE24106EAD51EE202D
:10577000116E126A136AD880D60E1054030E11549B
:10578000000E1254000E13541DE2D60E146E030EBA
:10579000156E166A176ADDDAEECF18F0EFCF19F042
:1057A0001A6A1B6A1850145C106E19501558116E45
:1057B0001A501658126E1B501758136E10C0ACF1C9
:1057C00011C0ADF1ACC1B0F3ADC1B1F3AAC1AEF33C
:1057D000ABC1AFF37CEC26F0BCDA0101AC51EE2694
:1057E000AD51ED22B6DA4FDA77DA01E305D8ACC174
:1057F000F3FFADC1F4FF12000301010EAB6F17EC14
:1058000026F0000903E1D7EC45F0F6D70101A051DD
:10581000140DF3CF57F7F4CF58F7000E07015727B1
:10582000010E58233ADA0C0E2ADA75DAF3CF4FF765
:10583000F4CF50F732DA0A0E22DA6DDAF3CF51F7ED
:10584000F4CF52F72ADA0E0E1ADAEECF53F7EFCF73
:1058500054F7080E07015327000E5423556B566B5F
:10586000140E0301CD6FCE6B18DA41DA53C799F4E9
:1058700054C79AF40401110E986F0FDA57C796F4C3
:1058800058C797F482EC4BF053C739F354C73AF337
:1058900010EC36F0F3CF53F7F4CF54F7080E0301B2
:1058A000B06FB16B03014F0EAE6F070EAF6F7CECA4
:1058B00026F0ACEC29F0F1D9120EE1D9EF68EDD960
:1058C0000E0EEB6A0F0EEB6A1200080E0101AE5DC0
:1058D0000AE2AEC1A0F134DAD880EE54000EED54E5
:1058E00001E3000C010C000C080E0101AF5D09E2A0
:1058F000AFC1A0F125DAC7D910C0F3FF11C0F4FF82
:105900001200F36AF46A120036DA01E1000CA051C9
:105910001CDAEF50010B01E032DAFCEC26F0B0C1EA
:10592000E9FFB1C1EAFFEF6E30DAEE06EF5A08DAAE
:10593000EE50ED1002E106EC28F0010C1CDA03E158
:10594000F36AF46A1200A05100DAEF50010B01E093
:1059500016DA1BDA98D9B451105CB551115805E22A
:10596000EFD9EECFB4F1EDCFB5F1B4C1B4F3B5C119
:10597000B5F3B2C1B2F3B3C1B3F336EC27F0F3CF52
:1059800041F7F4CF42F701DA07014151EE5E42518F
:10599000ED5AF1D902E106EC28F0B4C1F3FFB5C12C
:1059A000F4FF1200E8D902E006EC28F0EED9EE6A26
:1059B000ED6A1200080E0301B46FB56B0301460EC9
:1059C000B26F070EB36F36EC27F046C75DF747C7D7
:1059D00046F75DC747F748C75DF749C748F75DC752
:1059E00049F7080E106E07014B51D880105403E29E
:1059F0004A055D6F02D04AC75DF7080E4B5D4A6FDE
:105A00005DC74BF74C514D116AE04CC75DF74DC770
:105A10004CF75DC74DF7B6C1E9FFB7C1EAFF060E07
:105A20002ED9EECF4FF7EECF50F7EECF51F7EFCFA5
:105A300052F777D9EFCF53F7010E21D9EFCF54F7B3
:105A400070D9020E1CD9EFCF55F76BD9030E17D9B9
:105A5000EFCF56F7576B110E586FBAC159F7BBC14C
:105A60005AF7BAC139F3BBC13AF310EC36F0F3CFB1
:105A700059F7F4CF5AF70C0E0301416F426B030143
:105A80004F0E3F6F070E406F44EC36F0F3CF5BF7DD
:105A9000F4CF5CF707015B1F5C1F060E18D95BC7CC
:105AA000ADF35BEC26F0070E12D95CC7ADF35BECEF
:105AB00026F004019B6B9C6BF1EC4BF0BAC143F3F5
:105AC000BBC144F3B0EC36F0F3CF5BF7F4CF5CF737
:105AD00007014C51F3181CE14D515C1919E1B8C193
:105AE000C0F1B9C1C1F1B6C1BEF1B7C1BFF1010189
:105AF000460EBC6F070EBD6F22D807014E6F106EA9
:105B0000E0D809E1115007E1125005E1135003E11B
:105B100006EC28F0010C4E51A8D8100EB0D84AC798
:105B2000EEFF4BC7EDFF4E5110D9EF80010C010184
:105B3000A0519BD8E9CFF3FFEACFF4FF1200070191
:105B40000169000E026F010E036F006B080E005D0D
:105B50005BE2B2D80C0E0BD9020E91D8ECD8000142
:105B6000125010184AE11350111847E1A5D80A0E37
:105B7000FED8E1D8125010183EE1135011183BE145
:105B80009BD8100E7CD8EECF14F0EFCF15F0166A2C
:105B9000176A14501510161017102DE1BEC1E9FF39
:105BA000BFC1EAFF060E6BD8EECF10F0EECF11F0BA
:105BB000C2D882D8060E63D8EE50101808E1EE5015
:105BC000111805E1EE50121802E1EE50131810E022
:105BD000C0C1E9FFC1C1EAFFE868EE180CE1E8685E
:105BE000EE1809E1E868EE1806E1E868EE1803E14E
:105BF00007010051120000C701F70701140E022728
:105C0000000E0323002BA2D701C710F05AD805E1DC
:105C1000115003E1125001E1135024E00151140D21
:105C2000F3CF02F7F4CF03F7000E0227010E032390
:105C30000A0EE66EE66ABEC1E6FFBFC1E6FF3CD8CB
:105C400002C710F003C711F002C7E6FF03C7E6FF63
:105C500054D86CD818D830D80A0E10C0EBFF0B0EF1
:105C600011C0EBFF070101511200140DF3CFE9FF42
:105C7000F4CFEAFF000EE926010EEA221200E9261F
:105C8000000EEA221200EECF10F0EFCF11F012005A
:105C900041C7E9FF42C7EAFF120057C7E9FF58C7EB
:105CA000EAFF12005BC7E9FF5CC7EAFF120059C7B1
:105CB000E9FF5AC7EAFF120002C7E9FF03C7EAFF7C
:105CC0001200116A126A136AE868101812000401BF
:105CD0009B6F9C6BF1EF4BF0126A136AD60E105C4F
:105CE000030E1158000E1258000E13581200120E17
:105CF000EB500301CC6F21EF2AF0C0EC55F0126E8F
:105D0000060EE15E125012000301010EAC6F37EC7B
:105D100026F0E66E1200EECF39F3EDCF3AF310EF36
:105D200036F0B8C1E9FFB9C1EAFF1200BCC1E9FF12
:105D3000BDC1EAFF1200EECF12F0EFCF13F0120058
:105D4000A05193DF100E3FEF2EF08FDF130E3FEFC9
:105D50002EF09EDF0E0E3FEF2EF0A9DF0E0E3FEF6E
:105D60002EF0120E8CDFE552E750EF6E120087DF47
:105D70008ADF96EF2EF009D8EE50ED101200A051F8
:105D8000E4DFEF90080E67EF2EF00101A0EF2EF098
:105D900005010E5101E112007DDB05E1115003E127
:105DA000125001E1135002E0020E01D0010E0E6FFD
:105DB000116B0F9112006EDB05E1115003E11250DF
:105DC00001E1135001E053DB05010E6B6DDBFE0BAF
:105DD0004DEF32F005010E5108E166DB01095DDB94
:105DE0000501010E0E6F116B0F91120005010E518E
:105DF000080A01E1E1D0020A01E1DED0060A01E170
:105E0000DBD00B0A01E1C9D00E0A01E1C6D0020ABB
:105E100001E1C3D00D0A01E19DD0030A62E0010A4D
:105E200056E0070A42E0010A0EE0030A01E0120010
:105E3000FBDA07E1115005E1125003E1135001E1D3
:105E40001200020E0E6F1ADB01E112000A0EE66E5E
:105E5000E66AE66805011051140DF3CFE9FFF4CFAF
:105E6000EAFF000EE926010EEA22E9CF10F0EACFA0
:105E700011F0E9CFE6FFEACFE6FFEBEC55F0126E4A
:105E8000050EE15E125004013C0E486F496B4A6BEF
:105E90004B6B586B0501116B0F910F9304015E6BF7
:105EA0000401010E1DDB030E07D0B1DA07E287DA29
:105EB00001E2A5D00501020E0E6F120005010F854B
:105EC0009FD8020801E012000501040E0E6FD6DA19
:105ED00001E1120004015E6B0401030E01DB050EFB
:105EE00007D095DA07E26BDA01E289D00501020EEC
:105EF0000E6F120085D8060A29E0030A01E012009D
:105F0000B6DA7CDA060E0E6F0F81112B040158A150
:105F100008D04CC400F34DC401F34EC402F34FC487
:105F200003F358A508D054C40AF355C40BF356C460
:105F30000CF357C40DF358A30CD050C40EF351C446
:105F40000FF352C410F353C411F312000501020EF3
:105F50000E6F120034DA01E21200020E0401485DF5
:105F6000000E4959000E4A59000E4B590BE3640EBE
:105F70005927000E5A235B235C234807495B4A5B81
:105F80004B5B120051DA07E1115005E1125003E1B9
:105F9000135001E11200070E0E6F70DA01E11200DA
:105FA0000401010E5E6F0401030E5D6F57D90501F8
:105FB0000F9324DA0E2B12002ADA12E200DA1FE322
:105FC00005010E2B0C0EE76E0E19E8AE02D00E3551
:105FD00003D0E750D8800E5512E2020E0E6F120069
:105FE0000FD8060A08E0030A01E0120040DA06DAD8
:105FF000112B060E02D00501020E0E6F12001200C8
:106000000701036BD6D9020E0701005D01E0FFD046
:10601000016B0F0E015D02E257DAFBD705010FA3FA
:1060200007D00701016B040E015D08E24DDAFBD7D2
:106030002BDA4C0EB26F040E42DA58810701016B65
:10604000080E015D02E240DAFBD7016B060E015D2E
:106050000EE2AFD907010151EA6A040FE96E030E9F
:10606000EA22EF50005D01E0F6D0012BEFD7016B83
:10607000CE0E015D02E228DAFBD7046B9AD9000943
:1060800004E10701010E046FC2D007010051330A79
:1060900001E171D0CC0A6CE0C90A55E0350A2FE065
:1060A000020A18E0340A01E09DD083D907010005F7
:1060B00001E0D1D00101030EB06F070E0EDA050129
:1060C0000F51020B01E19DD0020E0701035D01E0BB
:1060D00098D0C1D0FDD901E0BED005010FA308D0F2
:1060E0000701016B040E015D01E38BD0EDD9FAD7F6
:1060F000CBD9540EB26F040EE2D9588582D001017B
:10610000020EB06F070EE9D9040E0701025D01E22D
:10611000A2D005010FA307D00701016B040E015D9A
:1061200008E2D2D9FBD7B0D9500EB26F040EC7D94E
:106130005883040E0701025F07010251020700099C
:1061400060E037D9F9D7C4D901E085D00101080E44
:10615000B06F070E7ED9070EB06F070E7AD9060E04
:10616000B06F070E76D9050EB06F070EB6D949D0BD
:10617000010E046F46D0ACD96EE105010FA307D024
:106180000701016B040E015D3CE29ED9FBD70101C2
:106190004B0EB06F040E5DD94A0EB06F040E59D984
:1061A000490EB06F040E55D9480EB06F040E95D944
:1061B00048C410F049C411F04AC412F04BC413F0A3
:1061C000050ED8901332123211321032E806F9E17E
:1061D00010500401485F1150495B12504A5B135044
:1061E0004B5B0FD00101020EB06F070E76D907018D
:1061F00002510207000905E00101000EB06F070E11
:10620000F5D7D7EC45F00701045101E137D7020E6D
:10621000035D0BE105C744F406C745F407C746F420
:1062200008C747F405010F8311D0440EE96E040E30
:10623000EA6EEE50051908E1EE50061905E1EE5040
:10624000071902E1EE50081901E0036BD2EC2CF0C3
:10625000070103511200D2EC2CF0000C0101010ED9
:10626000C8D8010EC6D8060EC4D84AD90101120EEC
:10627000C0D8230EBED8340EBCD8560EBAD8E5D836
:106280000101800EB6D83CD9030E04015D5D04E126
:106290005E5102E0E1D804D00101D7D80101D5D880
:1062A0000701006B0C0E005D02E204D9FBD7060E5D
:1062B0000101AC6FAD6B0101040EAA6F030EAB6F51
:1062C00089EC2BF00701006BCA0E005D02E2F2D8E8
:1062D000FBD70101630E8DD8820E8BD8530E89D85F
:1062E000630E87D8350E85D8010EA96F56EC2BF0BA
:1062F0005DC4A9F156EC2BF004015D0502E1050136
:106300000F93030E04015D5D15E15E5113E1010180
:10631000360EEBD847C4A9F156EC2BF046C4A9F1D0
:1063200056EC2BF045C4A9F156EC2BF044C4A9F16E
:1063300056EC2BF00101370E5CD8040E5AD8010E32
:1063400058D8030E56D8060E54D80C0EA96F56EC2A
:106350002BF0030E04015D5D02E15E5107E05D0577
:1063600009E14C514D114E114F1104E00101320E63
:10637000BCD872D80101A96956EC2BF000C301F713
:1063800001C302F702C303F703C304F704015E511C
:1063900005E10301006B016B026B036BFCEC2BF05E
:1063A00001C700F302C701F303C702F304C703F3F5
:1063B00012000101000EB06F070E6DEF32F0590EA2
:1063C000E96E040EEA6EEE500201F95D106EEE50B9
:1063D000FA59116EEE50FB59126EEE50FC59136EC5
:1063E000C80E105C000E1158000E1258000E135803
:1063F0001200A96F56EC2BF001011200F9C259F4FA
:10640000FAC25AF4FBC25BF4FCC25CF4120010C581
:10641000AFF174EC2CF0F3CF10F0F4CF11F0FA0ED2
:10642000F35C000EF4581200430E0101A56FA66B39
:106430000101A36BA46B440E0101A16FA26BEAECF6
:106440002AF00501106F106E55D05AD8010180EF67
:1064500032F043D801011200040E0101AC6FAD6BA4
:1064600001014C0EAA6F040EAB6F89EF2BF010C523
:10647000A7F137EC2BF005011069120010C5A8F147
:106480004AEC2BF000091200040E0101B46FB56B49
:106490000101120010C510F02DD0A86E160E0301D8
:1064A0002C6F2D6B53EF43F0160E03012A6F2B6BED
:1064B00042EF43F0010124D80701002B1200B36F13
:1064C0009EEC2CF00401120074DF0701012B120076
:1064D00070DF040E0701005D1200B16F84EF2CF035
:1064E0005D6FBCDE8BDF0501120083DF040EA96F38
:1064F00056EF2BF0116A126A136AE868101812003E
:06650000A96B56EF2BF021
:0A65060094909492949493809382F1
:106510009388938A0201010E916F926B936B8E6B3D
:106520008F6B906B946B07014F6B050E4F5D0EE206
:1065300032DBEE6AED6A2FDB020E3FDB2CDB040E52
:106540003CDB29DB060E39DB4F2BEFD70201C86B92
:10655000C96B0501066B076B0501086B096B12001F
:106560008150010B106E02018F51200B01E0010ED2
:10657000105C06E18150010B02E08F9B01D08F8BF4
:106580008150020B01E0010E106E8F51800B01E073
:10659000010E105C06E18150020B02E08F9F01D0DA
:1065A0008F8F8150100B01E0010E106E8F51100B78
:1065B00001E0010E105C06E18150100B02E08F99A2
:1065C00001D08F898150200B01E0010E106E8F5198
:1065D000400B01E0010E105C06E18150200B02E04F
:1065E0008F9D01D08F8D8050010B106E8E51800BCE
:1065F00001E0010E105C05E08E9F8050010B01E070
:106600008E8F8050020B01E0010E106E8F51020B35
:1066100001E0010E105C05E08F938050020B01E059
:106620008F838050040B01E0010E106E8F51080B18
:1066300001E0010E105C05E08F978050040B01E033
:106640008F878050080B01E0010E106E8E51400BB9
:1066500001E0010E105C05E08E9D8050080B01E00A
:106660008E8D8050200B01E0010E106E8F51010BBA
:10667000105C05E08F918050200B01E08F818050ED
:10668000100B01E0010E106E8F51040B01E0010EA2
:10669000105C05E08F958050100B01E08F858E0E09
:1066A000E96E020EEA6EEE50911905E1EE50921974
:1066B00002E1EE50931928E08B940701016B030E61
:1066C000015D18E2800E006F8B920151EA6A8E0F15
:1066D000E96E020EEA22EF50001502E08B8001D035
:1066E0008B908B82000503E18B92012BE8D7004150
:1066F0007F0BE9D78B848B94949A8B9A8EC291F2FC
:106700008FC292F290C293F29250010B19E050DACC
:10671000010E37DA15E18050010B36DA010E31DA5D
:1067200002E1000E01D0010E025D0AE005010881C0
:106730000701025103E00501068102D0050106911F
:106740009250020B1BE034DA020E1BDA17E1805084
:10675000020B01E0010E18DA020E13DA02E1000E5C
:1067600001D0010E025D0AE0050108830701025114
:1067700003E00501068302D0050106939250040B45
:106780001BE016DA040EFDD917E18050040B01E07E
:10679000010EFAD9040EF5D902E1000E01D0010E66
:1067A000025D0AE0050108850701025103E00501C9
:1067B000068502D0050106959250080B1BE0F8D91A
:1067C000080EDFD917E18050080B01E0010EDCD97B
:1067D000080ED7D902E1000E01D0010E025D0AE0D9
:1067E000050108870701025103E00501068702D071
:1067F000050106979250200B1BE0DAD9100EC1D983
:1068000017E18050200B01E0010EBED9100EB9D95E
:1068100002E1000E01D0010E025D0AE005010889C7
:106820000701025103E00501068902D0050106991E
:106830009250100B1BE0BCD9200EA3D917E1805059
:10684000100B01E0010EA0D9200E9BD902E1000E31
:1068500001D0010E025D0AE00501088B070102511B
:1068600003E00501068B02D00501069B9350010B46
:106870001AE09ED9400E85D916E18150010B010A1C
:1068800083D9400E7ED902E1000E01D0010E025DD7
:106890000AE00501088D0701025103E00501068D9C
:1068A00002D00501069D9350020B1CE081D9800E99
:1068B00068D918E18150020B020A01E0010E64D987
:1068C000800E5FD902E1000E01D0010E025D0AE0E8
:1068D0000501088F0701025103E00501068F02D070
:1068E0000501069F9350100B20E009C511F0126AB4
:1068F000136A106A010E5AD918E18150100B100A60
:1069000001E0010E60D9010E51D902E1000E01D063
:10691000010E025D0AE0050109810701025103E051
:106920000501078102D0050107919350200B20E05B
:1069300009C511F0126A136A106A020E37D918E1FC
:106940008150200B200A01E0010E3DD9020E2ED904
:1069500002E1000E01D0010E025D0AE0050109838B
:106960000701025103E005010783120005010793A7
:1069700012000701416B14C510F0010E02D95DE051
:1069800012C5A8F14AEC2BF0000957E0010E0701EF
:10699000436F446B426B0A0E425D4FE24351050167
:1069A0000815106E0701445105010915116E1050AC
:1069B00011103DE043C710F044C711F0101E111E26
:1069C0001050081711500917070141810101780E75
:1069D00002D9060E0701425D07E20101340EFBD821
:1069E000300E0701422507D00101320EF4D8300ED7
:1069F00007014225FA0F0101EED801013D0EEBD847
:106A00000501065107014315106E050107510701E5
:106A10004415116E1050111002E1300E01D0310EEC
:106A20000101D9D801013B0EA96F56EC2BF00701EB
:106A3000D89043374437422BAED70701415112005B
:106A4000F36AF46A12000701626B81A0628181A27D
:106A5000628381A8628581AA628762511200020165
:106A6000CB51040A31E0070A25E0010A19E0030AC4
:106A70000DE0010A01E01200CC518E93E8B08E8344
:106A8000CC519091E8A028D090811200CC518E97E3
:106A9000E8B08E87CC519093E8A01ED0908312006E
:106AA000CC518E9BE8B08E8BCC519095E8A014D041
:106AB00090851200CC518E95E8B08E85CC51909780
:106AC000E8A00AD090871200CC518E99E8B08E8948
:106AD000CC519099E8B0908912000201CD51050A7D
:106AE00042E0010A35E0070A28E0010A1BE0030A38
:106AF0000EE0010A01E01200CE518E9FE8B08E8FA9
:106B0000CE51E8B08980E8B037D089901200CE51DC
:106B10008F93E8B08F83CE51E8B08982E8B02CD053
:106B200089921200CE518F97E8B08F87CE51E8B08E
:106B30008984E8B021D089941200CE518E9DE8B0AE
:106B40008E8DCE51E8B08986E8B016D089961200B5
:106B5000CE518F91E8B08F81CE51E8B0898AE8B0EC
:106B60000BD0899A1200CE518F95E8B08F85CE5107
:106B7000E8B08988E8A089981200120002019051BB
:106B800012001016116A2AD00701026F06C510F014
:106B9000126A136A12004F51080DF3CFE9FFF4CFC8
:106BA000EAFFA00EE926020EEA221200111616D004
:106BB00008C510F0126A136A1200E926000EEA22D4
:106BC000EE6AED6A12000701026F07C511F0126A42
:106BD000136A106A1200A96F56EF2BF0126A136A3B
:0A6BE00010501110121013101200D3
:066BEA000F0E0301371736
:106BF0003751090804E2410E3725F60F1200300E16
:106C000037251200030138390F0B386FE850090897
:106C100004E2410E3825F60F1200300E382512001E
:106C20003AC3F3FF39C3F4FF12003BC301F73CC37F
:106C300002F73DC303F73EC304F70701010E056FDA
:106C4000070E066F05C7E9FFEA6E030ED0DAEF50B4
:106C5000E66E030EC6DA00C7EFFF93DA020EC7DA5C
:106C6000010EA6DAEF50E66E8CDA020EBADA010EE9
:106C70009FDA00C7EFFF01C704F002C705F003C7A2
:106C800006F004C707F012000701D16BD26BD36B7B
:106C9000D46B3FC3CFF740C3D0F741C3CDF742C356
:106CA000CEF7D890CE33CD33CDC710F0CEC711F08C
:106CB000CD07000ECE5B1050111018E0CFC7E9FFD2
:106CC000D0C7EAFF020ECF27000ED023EECF10F080
:106CD000EFCF11F0000110500701D1270001115032
:106CE0000701D223000ED323D423DED70301415161
:106CF000010B0EE0CFC7E9FFD0C7EAFFEFCF10F0DE
:106D0000000110500701D127000ED223D323D42332
:106D10000701D351D41119E0D1C710F0D2C711F037
:106D2000126A136AD3C714F0D4C715F0166A176A2B
:106D300010501424D16F11501520D26F125016200C
:106D4000D36F13501720D46FE3D7D1C710F0D2C739
:106D500011F0101E111E10C0F3FF11C0F4FF12003D
:106D60000701010E006F016B026B030143514411D7
:106D70005AE043C314F044C315F0166A176A400E74
:106D8000145C000E1558000E1658000E175804E338
:106D9000400E106E116A04D043C310F044C311F0CA
:106DA000126A136A10C005F7070110500301B46F8F
:106DB000B56B0301060EB26F070EB36F36EC27F00A
:106DC00007010551106E116A10500301435F115005
:106DD000445B0701046B0551045DC7E20451EA6A94
:106DE000060FE96E070EEA22EFCF03F700510AE122
:106DF00003510125016F0351015D0DE2022B0BE1EF
:106E0000012B09D003510225026F0351025D03E2F9
:106E1000012B01E1022B005102E0000E01D0010E16
:106E2000006F042BD8D70701021D026F011DF36EFE
:106E300002C7F4FF120003014551390805E3300E83
:106E4000455D02E3300E0FD04551460805E3410E83
:106E5000455D02E3370E07D04551660806E3610E33
:106E6000455D03E3570E455D1200FF0C010E030163
:106E7000EA6A4625E96E4751EA22EFCF45F3DBDFA8
:106E800007018D6F46C3E9FF47C3EAFFEFCF45F324
:106E9000D2DF07018E6FFF0E8D5D03E0FF0E8E5D6A
:106EA00001E1000C8E39F00B8D1148C3E9FF49C395
:106EB000EAFFEF6E010C07018D6BA6A203D0D7ECA1
:106EC00045F0FBD72F0EA616A68403014CC3E9FF9D
:106ED0004DC3EAFF4C2B000E4D23EF50A86E070167
:106EE0008D2B03014E510701D8808D5501E2A86A10
:106EF0004BC310F0116A1050AA6E03014AC310F080
:106F00004BC311F04A2B000E4B231050A96E550EA7
:106F1000A76EAA0EA76EA6820000A6A203D0D7EC89
:106F200045F0FBD7A850D1E1A69407018D0500D00C
:106F300012000701CD6BA6A203D0D7EC45F0FBD71A
:106F40003F0EA6160701CD2B030153510701D88030
:106F5000CD5506E24FC3E9FF50C3EAFFEF6A16D0F2
:106F600051C3A9FF52C310F01050AA6E0301512B58
:106F7000000E5223A680A8504FC3E9FF50C3EAFF7A
:106F8000EF6E4F2B000E5023A850DCE10701CD051A
:106F9000120057C310F01050AA6E56C3A9FF3F0E3F
:106FA000A616030154C3E9FF55C3EAFF542B000E94
:106FB0005523EFCF4FF7A680A85007014F5D01E0A2
:106FC000010C4F5101E1000CA92AEBE1AA2AE9D7F3
:106FD000030158C3E9FF59C3EAFF582B000E592398
:106FE000EFCFCDF7EF5024E0610E0701CD5D05E353
:106FF000CD517A0802E3200ECD5F03015AC3F6FF9C
:107000005A2B5BC3F7FF000E5B235CC3F8FF5C23C6
:107010000800F5500701CD5D01E0000C5AC3F6FFF2
:107020005BC3F7FF5CC3F8FF0800F550D1E1010C2A
:10703000000C5DC35CF75EC35DF707015A6B5B6BC9
:1070400003015F5107015A5D0301605107015B595C
:107050000BE25CC7E9FF5DC7EAFF5C2B000E5D2316
:10706000EF6A5A2B5B23ECD712001200030E0301C8
:107070006A5D3DE379D88AD813AE02D014681568EA
:10708000C1D8010E78D8EF380F0B166E89D81610BC
:10709000BCD813AE02D014681568B4D8060E176EAB
:1070A000020E69D8EF5017C0E7FFE75204E0E8424C
:1070B0007F0BE706FCE1166E010E03019DD816104A
:1070C000A4D813AE02D0146815689CD8020E53D809
:1070D000EF503F0B9AD813AE02D01468156840D811
:1070E000030E6827000E6923030E6A5FBFD76A513B
:1070F000000830E239D84AD813AE02D014681568B7
:107100002FD84ED80701CD6F03016A51010806E25E
:10711000010E31D8EF380F0B0701CD1325D8CDC79D
:1071200013F0146A156A48D8E66E030155D8020EAA
:107130006A5D02E23D0E09D017D8010E5DD865D810
:1071400013AE02D01468156837D8E66E45D861D8FA
:107150003D0EEF6E66C3E9FF67C3EAFFEF6A1200F8
:107160002BD8E66EECEF38F0F60E106EB80E116EFE
:10717000000E126E1200EA6A6825E96E6951EA2271
:10718000120005C7E9FF06C7EAFF120068C3E9FF5E
:1071900069C3EAFFEF50E840E8403F0B05EF39F0E4
:1071A00068C3E9FF69C3EAFFEF38F00B300B120048
:1071B000E926000EEA22120010501324F36E11503B
:1071C0001420F46E12501520F86EF4CFF7FFF3CFB1
:1071D000F6FF0800F55012001CD8E552E750EF6E9C
:1071E0001200E6DFE552E750EF6EC1EF38F0E0DF66
:1071F000EFCF00F7C1EF38F0BEDFEF50040DF350D2
:107200003C0B1200ADDFB4EF38F0136E146A156A50
:10721000120066C3E9FF67C3EAFF662B000E67230F
:0272200012005A
:0E7222000401CD5101E112000401030EF66FCC
:10723000B30EF76F000EF86F4EEC5AF00401260EF5
:10724000F66FB10EF76F000EF86F4EEC5AF0CDC42A
:10725000A9F70701A951000815E2A951070B05E19B
:1072600004012E0EF26F00EC5AF00201D95102E037
:107270006DD908D00B01320EFF6FA9EC5CF007014D
:10728000A907E7D704014E0EF66FB10EF76F000E97
:10729000F86F4EEC5AF00401000ECE6F030ECF6F64
:1072A00052EF39F05FDA0DDA010EE926000EEA221C
:1072B00008DA020EE926000EEA2203DA030EE926B6
:1072C000000EEA22A5EF3BF00701016B0201D95144
:1072D0001EE0ECEC59F00701006F0D0E005D1AE0A6
:1072E0000A0E005D17E0012B0401D0C4E9FFD1C4F0
:1072F000EAFFD02B000ED12300C7EFFFD0C4E9FF77
:10730000D1C4EAFFEF6AD251D207000903E0D7ECFB
:1073100045F0DCD7070101511200D3C401F7D4C4F2
:1073200002F70701036BD3C4E9FFD4C4EAFFEFCF30
:1073300000F7EF5021E02E0E0701005D11E104017E
:10734000D3C4E9FFD4C4EAFFD32B000ED423EF6AE1
:10735000D6D9032BEAD9D3C401F7D4C402F707D096
:10736000300E005D03E30051390801E2000C040116
:10737000D32B000ED423D7D7C2D9D7D9030E0701F8
:10738000035D01E0000C010C0201D95103E1D7ECCF
:1073900045F0FAD7ECEC59F00701006F310E005DB3
:1073A00005E3390E005D02E200511200390C0401C0
:1073B0000D0ED5D904010A0ED2D9300E0401D75DC5
:1073C000FF0F030DF3CFE9FFF4CFEAFF5F0EE926CD
:1073D000040EEA22EECFF6F4EECFF7F4EFCFF8F496
:1073E0004EEC5AF00401D751380A01E1AED00F0A31
:1073F00001E1A9D0010A01E19FD0030A01E198D07F
:10740000010A50E0070A47E0010A3EE0030A01E0F2
:107410001200330E85D90701A16F340E81D90701FF
:10742000A26F870EE66E070EE66EA1C7E6FFA2C743
:10743000E6FFA6D9870EF46F070EF56F3BEC5AF006
:1074400046D9000949E0870EE66E070EE66E92EC1B
:1074500054F0E552E552F3CFA1F7F4CFA2F7F3CF02
:10746000A8FF330E47D9A2C7A8FF340E43D9A2C73D
:10747000A8FF080E3FD9A1C7A8FF090E3BD9A2C794
:1074800008F3A1C709F312000701000E9F6F030E56
:10749000A06FA36B0ED007010E0E9F6F030EA06F9F
:1074A0000E0E06D007010A0E9F6F030EA06F0A0E84
:1074B000A36F9FC7CEF4A0C7CFF4F4DE08D90401B0
:1074C0009B0ED56F070ED66F0401870ED36F070E84
:1074D000D46F23DF000911E10401B90EF66FB20E7B
:1074E000F76F000EF86F4EEC5AF00201D95103E12C
:1074F000D7EC45F0FAD7ECEF59F09FC7E9FFA0C7EA
:10750000EAFF9BC7EEFF9CC7EEFF9DC7EEFF9EC73D
:10751000EEFF9BC7A8FF2FD99CC7A8FF2CD99DC7FA
:10752000A8FF29D99EC7A8FF0701A351A32B09D003
:10753000160EF6D8010903D0160EF2D8FE0BA86E6F
:10754000160E7AEF3BF0BFEF3AF012000401830E03
:10755000F66FB10EF76F000EF86F4EEC5AF014DFB5
:107560000701AA6F390EAA5D03E0AAC7D7F41FDF8F
:10757000D7EC45F0380E0701AA5DE8E112000701DB
:10758000006B026BE1EC3FF0F9C285F7FAC286F7B7
:10759000070185510201F95D106EFA510701865508
:1075A000116E320E105C000E115809E3F9C285F716
:1075B000FAC286F70401150EF26F00EC5AF0D7EC10
:1075C00045F00201D951E4E00701025101E078D011
:1075D000D7EC45F00201D951F7E0ECEC59F0070186
:1075E000016F0051030A2FE0010A2AE0030A23E099
:1075F000A6D8010E101808E1115006E1125004E15E
:10760000135002E1010E1DD09AD8040E10180FE19C
:1076100011500DE112500BE1135009E129EC40F03B
:107620000401060E9CD80701010E026FCDD704019C
:10763000150E95D8C9D7060E046F036B020E01D044
:10764000030E006FC1D70351032BEA6A050FE96EE1
:10765000070EEA2201C7EFFF03C710F0116A126A92
:10766000136AD880800E1054000E1154000E12546C
:10767000000E1354A9E2060E046F016B60D8800E51
:10768000105C000E1158000E1258000E13580DE237
:107690000151EA6A050FE96E070EEA22EFCF8DF27B
:1076A000FCEC3FF00701012BE9D702017F6B2DECC9
:1076B0003FF004C7F2F400EC5AF00701006B84D7E6
:1076C000010C43D804012E0E4AD8B2EF3BF004015E
:1076D000290E45D804013A0E42D80401200E3FD8A5
:1076E0000401140ED26F0401870ED06F070ED16F04
:1076F00064EF39F003012C6F2D6B53EF43F001C79A
:10770000E6FF02C7E6FF92EC54F0E552E552F35073
:10771000E66ED5C410F0D6C411F007010351120073
:1077200003012A6F2B6B42EF43F00F011024E96E27
:10773000000E1120EA6EE552E750EF6E120001C70D
:1077400010F0116A126A136A1200EF50E66EE66AD0
:1077500017D8000EF46F070EF56F3BEF5AF0F26F7B
:1077600000EF5AF0000EE66E070EE66ECEC4E9FF9B
:10777000CFC4EAFF12000701A351A32B7AEF3BF01D
:1077800007EC55F0E552E552E552E55204011200CE
:10779000150E0001B36FB46B37EC12F00201016FEC
:1077A000056B336B006B140E036F046B120001C288
:1077B000B9F001EC13F0000908E10201336B080E87
:1077C000076F056B006B066B010C01C2D2F0D6ECA3
:1077D00015F0000940E05EDA0001700ED06F070E70
:1077E000D16F01C2CFF097EC15F000091AE0020149
:1077F0003351332BEA6A120FE96E020EEA2270C788
:10780000EFFF33C210F0116A126A136A1F0E1018CC
:10781000E3E11150E1E11250DFE11350DDE1336BA0
:10782000DBD701C2C4F0BBEC14F00A0E0701705D97
:1078300027E102013351EA6A120FE96E020EEA22D1
:10784000EF6A336BC3D934C246F235C247F28CD9E2
:107850000201076F15D00201055112E043510201E8
:10786000F95D106EFA5102014455116E500E105C14
:10787000460E115805E30EDA020E076F010E056F72
:1078800002010551010A3DE0050A04E0040A57E13E
:10789000086B00DA01C2BCF0A3EC13F0000901E1AF
:1078A000010C08C2E9FFEA6AE9BEEA68DDD9D70E31
:1078B000E926010EEA22EECF71F7EECF72F7EFCF95
:1078C00073F7070171C7F6FF712B72C7F7FF000E40
:1078D000722373C7F8FF73230800F5CF70F7F550D4
:1078E00007E070C7BEF001C2BDF0CEEC13F0E9D7DF
:1078F00001C2BBF04DEC13F002010C0E086F010E3B
:10790000056F080E075D1BE007C245F219D8000994
:107910000FE00C0E0201085D03E0040E056F04D0B9
:10792000020E075D01E1056B080E076F066B010C87
:107930000C0E0201085D03E0040E056FABD7010CCD
:1079400002014551060A54E0030A50E0060A4CE0E1
:10795000070A34E0060A30E0030A18E0010A59E198
:1079600000810093010E086F090EE66EE66A36C2CA
:10797000E6FF37C2E6FF090EE66E020EE66E62EC27
:1079800056F0106E060EE15E1050010C00A112D0F0
:1079900036C2CBF437C2CCF40401090EC96F020E13
:1079A000CA6F28EC47F0000904E002010083020ED0
:1079B00031D00201060E2ED00CEF3DF03EC2E6FFA4
:1079C0003FC2E6FF92EC54F0E552E552F3CF04F2E9
:1079D00040C2E6FF41C2E6FF92EC54F0E552E552A8
:1079E000F3CF03F2020102D03FEF3DF00B0E12D0B5
:1079F0000B0E086F02C210F041D905E1115003E1EE
:107A0000125001E1135007E002C2BAF00AEC13F081
:107A1000010C050E086F010C02010651030A1EE05D
:107A2000020A15E0010A2AE1020E065D02E129ECD4
:107A300040F002C210F022D905E1115003E11250CA
:107A400001E1135006E030D90201010E05D01CD926
:107A500015E10201030E086F066F000C01C2BCF0B5
:107A6000A3EC13F000090AE001C2B9F001EC13F035
:107A7000000904E001C2BAF00AEC13F0000C0201A4
:107A80000651020A45E0030A2CE0010A6CE100B34A
:107A900002D0060E66D0070E086F03C2B7F004C20C
:107AA000B8F00151240DF3CFE9FFF4CFEAFF000E47
:107AB000E9260A0EEA22EE52E9CFB5F0EACFB6F097
:107AC00085EC12F00201026F106ED8D805E111505A
:107AD00003E1125001E1135002E0010E17D00A0E2B
:107AE00040D0D2D840E079C210F0116A126A136A0D
:107AF000010E1016116A126A136A1050111012103A
:107B0000131031E0E1EC3FF00201020E066F000CB1
:107B100002C2D2F0D6EC15F000091CE0BBD800017F
:107B2000740ED06F070ED16F02C2CFF097EC15F034
:107B3000000907E074C78DF2FCEC3FF0D7EC45F08C
:107B4000EED702017F6B2DEC3FF002C2C4F0BBEC1C
:107B500014F0000C99D807E1A7D80201FE0E026FBD
:107B6000090E086F010C000C0701006B070EE76E91
:107B70000019E8AE02D0E73402D0E750005D25E2FC
:107B8000040EE66EE66A00C7E9FFEA6AE9BEEA6843
:107B90006BD8C20EE926010EEA22EECFE6FFEECF49
:107BA000E6FFEFCFE6FF46C2E6FF47C2E6FFA1ECE5
:107BB00055F0106E070EE15E1050000903E1070159
:107BC000005112000701002BD1D7070C0701036BEE
:107BD000120E006F020E016F62D8EF50200804E110
:107BE000002B000E0123F8D700C734F201C735F28D
:107BF0000201010E426F53D8EFCF02F7EF5033E08E
:107C000007010351010A16E0010A29E1200E025D75
:107C100003E02C0E025D05E142D8EF6A010E036F0E
:107C20001ED00D0E025D03E00A0E025D18E137D88A
:107C3000EF6A15D0200E025D12E002014251422B84
:107C4000E96EEA6AD890E936EA36340EE926020E81
:107C5000EA2200C7EEFF01C7EDFF0701036B002B0F
:107C6000000E0123C8D71200030EEA02F3CFEAFF89
:107C7000E902F3CFE9FFF450EA261200116A126A12
:107C8000136AFE0E1018120002C2B9F001EC13F0D4
:107C900000091200F9C243F2FAC244F2120000C70E
:107CA000E9FF01C7EAFF120029EC40F002C2BAF076
:047CB0000AEF13F0D4
:0C7CB4000201786B010E796F0401180EBC
:107CC000B06FA5EC56F00701006B00C710F036DA74
:107CD000060ED3D905E20051D8D9EF6A002BF5D7AB
:107CE000010C0701FE0E026F79C210F034DA01E1D7
:107CF000FE0C016BF4D9060EC0D908E2015139DA45
:107D000003E101C702F702D0012BF4D702C710F03C
:107D100015DAFE0E101807E1115005E1125003E1CB
:107D2000135001E1FE0C450E036F046B056B7BC223
:107D3000E9FF7CC2EAFFEF5001E1FF0C7BC2E6FFE6
:107D40007CC2E6FF90EC56F0E552E552F3CF7BF2B1
:107D5000F4CF7CF203C7B5F404C7B6F4D1D904E07C
:107D60000701FE0E026F6CD02FEC57F00701006F79
:107D7000106EE4D9800E71D902E0026961D0016B06
:107D8000AED90C0E7AD922E22FEC57F00701006F22
:107D900001510201EA6A7B25E96E7C51EA22EF502B
:107DA0000701005D06E0120E0327000E04230523E1
:107DB0000DD0005109E10701012B91D90C0E5DD9BD
:107DC00005E22FEC57F0F7D7012BDAD788D90C0E44
:107DD000101831E111502FE112502DE113502BE119
:107DE0000251080DF3CF06F7F4CF07F7480E062728
:107DF000020E0723A7D9010EEF6EA4D9EB6A020E7B
:107E0000EB6A2FEC57F0E66E9DD9030E2DD9030EC9
:107E10009ED9010E29D9030E9AD9020E25D9060E34
:107E200023D9060E94D9010E92D9E552E750EF6E90
:107E30000201782B05D036EC57F0D7EC45F08AD705
:107E400036EC57F00701025112007EC27FF205D8CE
:107E500002017E511AD9EF6A120002017F51080D0A
:107E6000F3CFA4F7F4CFA5F7480E0701A427020E1D
:107E7000A5235BD9EF50106E126A136A6FD903E025
:107E800036EC57F010D051D92ED96BD90CE025EC37
:107E900057F00401A00EBE6F6FEC57F0000903E02D
:107EA000D7EC45F0F6D7F90E106E3FD9E850EF1633
:107EB00002017993120002018051080DF3CF01F7FE
:107EC000F4CF02F7480E07010127020E02239F0E8E
:107ED000E6D8E850EF16E3D806D93DD915E0DFD84B
:107EE00002D93CD914E140D90FE1D9D810D9D7D85B
:107EF000E0D810C0B5F411C0B6F402D905E1CFD86E
:107F0000EF820201798303D0CAD8EF8A000C2FECEC
:107F100057F00701006FC3D8EAD8C1D8D6D805E119
:107F20001350111802E1BBD8EF8C07010051120069
:107F3000010C02018151080DF3CF00F7F4CF01F7D6
:107F4000480E07010027020E0123AED8EF50106E35
:107F5000126A136A06D903E012D901E3EBD8A4D858
:107F6000C2D8FFD815E100D903E09ED8EF8A000CF3
:107F70009BD8CDD899D89DD810C0B2F411C0B3F415
:107F8000CDD805E191D8EF840201798301D0000CAE
:107F900082C2B7F411EC57F087D8A9D885D895D804
:107FA00005E11350111802E17FD8EF8C010C12008B
:107FB0001200F36AF46A1200056A066A076A120080
:107FC000000C79C210F0C7D801E1000C0701A46BC6
:107FD000A4C710F0B3D8060E50D806E2A451C9D8F1
:107FE00001E0000CA42BF4D70201010E486F400EF3
:107FF0004B6F4C6B4D6B010C0701480EA66F020EC8
:10800000A76F48C210F0ADD803E0B9D801E392D809
:1080100048C210F093D8A5D811E1A6D803E0020118
:10802000488B000C4BC2B2F44CC2B3F477D805E1D4
:108030000201488579837A6B01D0000C8DC2B7F4B8
:1080400011EC57F002017A2B4B2B000E4C234D23E1
:10805000010C70D80201486B010C10166FD810503B
:10806000111012101310120072D8E552E750EF6E83
:108070002FEC57F0E66EA2EF40F0105C000E1158A6
:10808000000E1258000E13581200080DF3CFE9FF2E
:10809000F4CFEAFF480EE926020EEA22120001C7D9
:1080A000E9FF02C7EAFF120000C7E9FF01C7EAFFC4
:1080B0001200030E4CD8EE501324106EEE50142014
:1080C000116EEE501520126E1200060E40D8EECF43
:1080D00012F0EFCF13F0000112501018120001C778
:1080E00010F09EEF40F0EF50106E9EEF40F0EE5219
:1080F000EE2A000EED22EECF10F0EDCF11F01200BF
:108100000401A00EB46FE4EC56F000091200EE5228
:10811000EECF13F0EFCF14F0156A12000401A00E99
:10812000B16FAEEC56F000091200A4C7E9FFA5C775
:10813000EAFF120002017F6B2DEF3FF0116A126A15
:10814000136A120006C7E9FF07C7EAFF1200E92613
:10815000000EEA221200010E2DEF40F0020E2DEF6C
:1081600040F0040E2DEF40F079C210F0E7DFAEEFE3
:1081700040F08BDFEFCF10F0E1DFABEF40F07AC2E1
:0A81800010F0DCDF400E3DEF40F090
:06818A00290EC2D904D841
:1081900084EC59F008EF5BF00701506B516B240E33
:1081A000B8D907014F6B030E4F5D1BE2C0D942ECFB
:1081B00043F0E66E07010DDAE552E750EF6E09DA9B
:1081C000D3D9B5D92A27000E2B2342EC43F0E66E13
:1081D000070104DAE552E750EF6E00DAC5D94F2BFC
:1081E000E2D750C710F051C711F0126A136AD88055
:1081F000000E1054020E1154000E1254000E1354AF
:108200001CE20201640ED46FDA6FE06BE66BEC6B7C
:10821000F26B07014F6B030E4F5D0FE2DAD96DD998
:1082200053EC43F00701DAD968D92C27000E2D232F
:1082300053EC43F007014F2BEED70201000ECF6F36
:10824000080ED06FD451CF25D56F000ED021D66F38
:10825000DA51D525DB6F000ED621DC6FE051DB252E
:10826000E16F000EDC21E26FE651E125E76F000EC1
:10827000E221E86FEC51E725ED6F000EE821EE6F8B
:10828000F251ED25F36F000EEE21F46F12000A0E8D
:1082900003015F6F606B0301500E5D6F070E5E6F31
:1082A00019EC38F00301120EFED807014F6F4FA1F1
:1082B0001AD0A4D926E1115024E1125022E1135022
:1082C00020E13FD9110EEFD857D9100EECD808D9BC
:1082D0000501206F106EECD814E1115012E112501C
:1082E00010E113500ED08AD905E1115003E112506C
:1082F00001E1135006E020C5A7F137EC2BF0050192
:1083000020690301150ECFD807014F6F4FA11AD076
:1083100079D917E1115015E1125013E1135020E102
:1083200010D9140EC0D828D9130EBDD8D9D805013C
:10833000216F106EBDD805E1115003E1125001E12B
:10834000135012005FD905E1115003E1125001E111
:10835000135006E021C5A7F137EC2BF00501216988
:1083600012000301160E9FD80701026FE85035E195
:1083700045D905E1115003E1125001E113502DE000
:1083800020C5AEF165EC2CF0000916E097D8800B03
:1083900011E0E1D80BE018D904E1C5D8D7EC45F0DD
:1083A000FAD703D901E11FD921D9F3D787D8020B16
:1083B00001E1B9D8D2EC2CF030D90FE020C5A8F1FA
:1083C0004AEC2BF0000909E028D905E0DDD801E1ED
:1083D00012D927D9F9D7FCEC2BF00301170E63D87B
:1083E0000701026FE85035E10DD905E1115003E1B5
:1083F000125001E113502DE021C5AEF165EC2CF0D7
:10840000000916E05BD8800B11E0A5D80BE0DCD8A2
:1084100004E189D8D7EC45F0FAD7C7D801E1E3D811
:10842000E5D8F3D74BD8020B01E17DD8D2EC2CF084
:10843000F4D80FE021C5A8F14AEC2BF0000909E0BF
:10844000ECD805E0A1D801E1D6D8EBD8F9D7FCECFF
:108450002BF00701026B030E025D04E264D80701F2
:10846000022BF9D712000201F851020A0BE0030AAD
:1084700006E0010A01E008D0D6EC59F005D00BEC7B
:108480005BF002D0000000D012000C0DF3CFE9FF2A
:10849000F4CFEAFFCF0EE926020EEA221200E92607
:1084A000000EEA2212002A6F010E2B6F42EF43F0FA
:1084B000116A126A136AE868101812000701025163
:1084C000EA6AF50FE96E020EEA22EF501200105030
:1084D000EE24E76E1150EE20EA6EE7CFE9FF1200BE
:1084E000E552E7CF11F0E552E7CF10F0010110108F
:1084F000A16F11C0A2F1EAEF2AF0EF50A86E4F5120
:10850000E82403012C6F2D6B000E2C27010E2D2368
:10851000120003015F6F606B0301CF0E5D6F020EEF
:108520005E6F19EF38F002C7F8F233EF42F04F51A7
:10853000E82403012A6F2B6B000E2A27010E2B2340
:1085400012000101A56BA66B0101500EA36F070E6F
:10855000A46F030112000101000EB06F070EB16F8E
:1085600084EC2CF000091200EF50106E116AE850F4
:108570005027115051231200106E116E106A10C056
:10858000E6FFE66E0301120052D8EF50106E116A3A
:108590003DD8060E84DF9BDFEFCF00F748D8EF2AE7
:1085A000EFCF10F033D80B0E34D045D8EF50106E0B
:1085B000116A2CD88CDF00C7EFFF3DD8EF2A3FD0DF
:1085C00025D80A0E4FEF42F0070120D8040E67DFCE
:1085D00036D04F515ADF050E4FEF42F04F5155DF65
:1085E0000B0E4FEF42F027D8EF6A12000FD8040E9F
:1085F00056DFEF2A12001BD8EF6A120020C510F0D8
:1086000058EF42F021C510F058EF42F0025145EF0B
:1086100042F045DFEF50105C12000701D1DFEF5050
:108620001200CEDFEF0600C7A9F156EF2BF0EEDF08
:10863000090E4FEF42F0EADF020E4FEF42F0EFCFAC
:0886400010F0E4DF050EE5D7A0
:08864800AA6AA96A3F0EA616FA
:108650000701000E006F030E016FA950106E116A22
:10866000120E105C000E11580CE2A68000C7E9FF44
:1086700001C7EAFF002B000E0123A8CFEFFFA92AB4
:10868000ECD712002AC3A9FF2BC310F0116A1050B7
:10869000AA6EA6A203D0D7EC45F0FBD73F0EA616D4
:1086A000A680A8501200A8CFA4F72CC3A9FF2DC301
:1086B00010F0116A1050AA6EA6A203D0D7EC45F0B4
:1086C000FBD73F0EA616A6800701A451A85C01E1C6
:1086D00012D0A4C7A8FF2F0EA616A684550EA76E0B
:1086E000AA0EA76EA6820000A6A203D0D7EC45F082
:1086F000FBD7A69400D012001200200EBBD90701B0
:10870000516F51A14CD0AC84080E7E6E1F0EB2D9B1
:10871000080A36E00F0A32E0010A2AE0030A23E0E1
:10872000010A1CE0070A15E0010A0EE0030A07E04F
:10873000010A28E10701340E4F6F820E1DD0070198
:108740008C0E4F6F200E18D00701450E4F6F100E84
:1087500013D00701220E4F6F080E0ED00701100E26
:108760004F6F040E09D00701080E4F6F020E04D0A0
:108770000701030E4F6F010E506F08D0AC0E03D0EF
:10878000560E01D0AC0E07014F6F506B4FC7AFFFB5
:1087900050C710F0116A10507F6E8BEF59F092EFB6
:1087A00059F01200230E66D9926E240E63D9070188
:1087B0004F6F7ED904E1330E07014F1305D07CD9EA
:1087C00003E1CF0E07014F174FC793FF250E52D974
:1087D000D80907014F6F6CD902E1D80E03D06CD9CC
:1087E00003E1F80E07014F174FC794FF280E42D937
:1087F000976E290E3FD91009986E12002A0E3AD9A9
:10880000896E2B0E37D98A6E2C0E34D90701006F72
:108810004FD902E10701008B00C78BFF2F0E2AD929
:108820008E6E300E27D98F6E1200310E23D9C16E95
:10883000320E20D98009C06E1200010E03012E5D98
:1088400046E32E51020801E2120031510DE02FC320
:10885000A8FF2E05E824660F12D930C3A8FF030134
:108860002E05E824670F0BD903012E050DD9EECF95
:108870008DF7EDCF8EF78DC78FF78EC790F7070175
:10888000010E8F5F000E905B060E0301D8902F370C
:108890003037E806FBE103012F51E840E8403F0B89
:1088A000300B106E8FC7E9FF90C7EAFFEF50CF0B78
:1088B00010100701916F8DC7E9FF8EC7EAFF30C323
:1088C000EFFF8FC7E9FF90C7EAFF91C7EFFF1200E4
:1088D0000701666B676B010E0301325D03E33251E2
:1088E000020803E2F36AF46A12003205CDD8EECF33
:1088F00062F7EDCF63F762C764F763C765F70701F7
:10890000010E645F000E655B62C7E9FF63C7EAFFA3
:10891000EF50666F676BD89066376737D8906637C9
:10892000673764C7E9FF65C7EAFFEF50300BE838E7
:108930000F0B661366C7F3FF67C7F4FF120033C35C
:108940008DF70301345104E08DC7A8FF640E97D85A
:10895000CB50106E116AFF0E101801E1115002E0A9
:10896000000E01D0010E010808E1030E07018D5D24
:1089700002E18D6B0BD0020E06D007018D5102E192
:10898000020E03D0030ED8808D558D6F030E8D1708
:10899000FC0ECA168D51CA121200030ECA1407012A
:1089A000626F030E625D01E16207CB50106E116AC7
:1089B000FF0E101804E1115002E1020E01D0030E67
:1089C000D880625512000301365104E035C3A8FF78
:1089D000630E55D8030135A103D00C0EBD1202D091
:1089E000F00EBD1635A303D00C0EBA1202D0F00E55
:1089F000BA16355102E0CA841200CA941200630EFE
:108A000039D8000901E11200B70EB116650E32D84F
:108A1000010B02E0CB6802D03F0ECB6E0301346B3A
:108A2000640E28D80301336F8ADF660E23D807014E
:108A30004F6F670E1FD832D8010E2E6FFEDE680E04
:108A400019D807014F6F690E15D828D8020E2E6F5E
:108A5000F4DE0301366B630E0DD80301356FE3EFCF
:108A600044F02AD802E1B8EF50F022D802E183ECBA
:108A700032F0120003012A6F2B6B42EF43F0030127
:108A80002C6F2D6B53EF43F0030DF3CFE9FFF4CFC1
:108A9000EAFF000EE926050EEA2212000701506FD8
:108AA0000301316B4FC72FF3E8CF30F303011200FE
:108AB000870EE0DF02081200870EDCDF01081200DB
:108AC000DACFE4FFE2CFDAFFE9CFE4FFEACFE4FF59
:108AD000F6CFE4FFF7CFE4FFF8CFE4FFF5CFE4FFF4
:108AE000F3CFE4FFF4CFE4FFFACFE4FFFBCFE4FFE2
:108AF00000EE00F0100EE80403E3EECFE4FFFBD736
:108B000000EE10F0100EE80403E3EECFE4FFFBD715
:108B1000E652F2A414D09E0ED76E580ED66E020105
:108B2000F92B000EFA23FB23FC230201FF0706E1C9
:108B3000640EFF6F0201FD2B000EFE23F2949E5087
:108B4000200B05E09D50200B02E0A6EC59F09E5052
:108B5000100B05E09D50100B02E0C5EC59F0E552FA
:108B600000EE1FF0100EE80403E3E5CFEDFFFBD7A6
:108B700000EE0FF0100EE80403E3E5CFEDFFFBD7A6
:108B8000E5CFFBFFE5CFFAFFE5CFF4FFE5CFF3FF3D
:108B9000E5CFF5FFE5CFF8FFE5CFF7FFE5CFF6FF2F
:108BA000E5CFEAFFE5CFE9FFE5CFDAFF1100CD9E83
:108BB000CFAE0FD00401C0510BE00401C06BFF0E1B
:108BC0000401BF5D05E00401BF5102E00401BF07DD
:108BD00003D00401010EC06F0401BF5101E0040085
:108BE00012000401010EC16FD180BF694BD9E6ECC0
:108BF0005CF0C5EC40F003012A6B2B6B42EC43F0B8
:108C0000000902E07DEC43F0F28EF28C5AEC3EF06B
:108C1000A0EC57F024EC43F0FEEC43F0D2EC43F030
:108C200015EC44F0FFEC44F0140E34D90401CD6F80
:108C300011EC39F019EC49F031EC45F04CEC4FF007
:108C400094EC1EF0C8EC3BF047EC41F018EC52F00D
:108C50006AEC04F021EC5DF00401260EBF6F150EE6
:108C600019D9020B20E005010B510201F95D106ECC
:108C7000320E105C18E3F9C20BF5240E0BD9400B31
:108C80000AE0240E07D9BF0BA86E240E03012C6F37
:108C90002D6B53EC43F0939C8A7C870EFBD8020823
:108CA00002E102018E715FEC4FF05BEC49F0A6EC43
:108CB00004F055EC52F0B1EC41F03BEC5CF0CBEC45
:108CC0001EF0D7EC3BF0CDEC4DF008D805010A5171
:108CD0000501115DC1E011C50AF5BED705010C51B2
:108CE0000201F95D106E010E105C0DE3F9C20CF586
:108CF000870ED0D8020A05E0030A05E1D6EC50F051
:108D000002D0B0EC32F005010D5119E10401C22B83
:108D10000C0EC25D01E3C26BC11C0F0BC25D0CE205
:108D2000C30EC216C251040DF350C212C280C282D9
:108D30000501010E0D6F03D0B2D8EE6AED6A050190
:108D40000D5114E0C250020B11E1C450136E126AAF
:108D5000C35000011210106E13C011F004019FD80F
:108D600010C0EEFF11C0EDFF05010D6B12000301F5
:108D7000140E5A6FBA0E5B6F000E5C6FC5C458F3C9
:108D8000C6C459F3E8EC37F0000961E00301080EAE
:108D9000536F350E0301516F526B0301880E4F6FF5
:108DA000070E506F99EC37F00701876FE850872B5B
:108DB000EA6A880FE96E070EEA223A0EEF6E0301A7
:108DC000080E536F3E0E0301516F526B070187511E
:108DD00003014F6F506B880E4F27070E502399ECFD
:108DE00037F0880EE66E070EE66E54EC56F0E5524C
:108DF000E552F3CF6AF30301880E686F070E696FBF
:108E000003019C0E666F070E676F36EC38F09C0E00
:108E1000E66E070EE66E150E0401116AC525106E8A
:108E2000C651112210C0E6FF11C0E6FF05EC56F056
:108E3000E552E552E552E552000909E1C3C4E9FFF4
:108E4000C4C4EAFF090EE926000EEA22EF841200EC
:108E5000350E0301566F576BC9C454F3CAC455F39A
:108E6000C9EC37F000090DE13E0E0301566F576B58
:108E7000CBC454F3CCC455F3C9EC37F0000901E17D
:108E8000010C000C070EB46EB10ECD6ECD9EF18EAE
:108E9000D56A120003012A6F2B6B42EF43F0C251D7
:108EA000E96EEA6AD890E936EA36120EE926030E30
:048EB000EA221200A0
:0C8EB40043616368652D436F6E74726F3C
:108EC0006C3A206D61782D6167653D3630302C201D
:108ED0006D7573742D726576616C69646174650D6E
:108EE0000A00485454502F312E3020343031205550
:108EF0006E617574686F72697A65640D0A575757A9
:108F00002D41757468656E7469636174653A2042B9
:108F100061736963207265616C6D3D226465666191
:108F2000756C74220D0A0D0A41757468656E74695A
:108F3000636174696F6E2052657175697265642131
:108F40000D0A00485454502F312E30203530332034
:108F50000D0A0D0A5365727669636520556E617658
:108F600061696C61626C650D0A00485454502F3180
:108F70002E3020343034204E6F7420666F756E644E
:108F80000D0A0D0A4E6F7420666F756E642E0D0A01
:108F900000617564696F2F782D7761766500617067
:108FA000706C69636174696F6E2F6A6176612D619F
:108FB00072636869766500696D6167652F6A7065BF
:108FC0006700696D6167652F67696600746578740D
:108FD0002F6A617661736372697074007465787466
:108FE0002F637373006170706C69636174696F6E75
:108FF0002F6A6176612D766D00746578742F6874C0
:109000006D6C00746578742F706C61696E000D0A68
:109010004E6F772072756E6E696E67206170706C2E
:1090200069636174696F6E2E2E2E000D0A526561A0
:10903000647920746F20646F776E6C6F6164204672
:10904000696C652053797374656D20496D6167653E
:10905000202D2055736520586D6F64656D207072EA
:109060006F746F636F6C2E0D0A000D0A44484350F5
:10907000202620495020476C65616E696E67206428
:10908000697361626C65642E0D0A000D0A444843E1
:1090900050202620495020476C65616E696E67201C
:1090A000656E61626C65642E0D0A000D0A4465668A
:1090B00061756C74205375626E6574204D61736BBD
:1090C0002028000D0A44656661756C742047617440
:1090D0006577617920416464726573732028000D9F
:1090E0000A44656661756C7420495020416464725D
:1090F0006573732028000D0A53657269616C204EF8
:10910000756D626572202800323030204F6B0D0A79
:10911000003432352043616E2774206372656174B8
:1091200065206461746120736F636B65742E202009
:10913000496E637265617365204D41585F534F43BB
:109140004B4554532E0D0A00323236205472616E54
:109150007366657220436F6D706C6574650D0A00EF
:1091600031323520446F6E650D0A003135302054A0
:1091700072616E7366657272696E67206461746194
:109180002E2E2E0D0A00353330204C6F67696E206D
:1091900072657175697265640D0A00353032204E52
:1091A0006F7420696D706C656D656E7465640D0A11
:1091B00000353030200D0A00323231204279650D01
:1091C0000A00323330204C6F6767656420696E0D8A
:1091D0000A003333312050617373776F72642072E9
:1091E000657175697265640D0A003232302052650E
:1091F0006164790D0A0041424F52005459504500B4
:10920000504F52540053544F52005155495400503E
:1092100041535300555345520047756573740059C7
:109220006573006C34303D323B006C34303D313B73
:01923000003D
:01923100003C
:0E9232000701006B00C710F05FD908E2005181
:1092400068D9EF6A00516BD9EF6A002BF4D712008E
:10925000C750040B01E0010E72D9FAE1C580C5B018
:10926000FED70401305143D9C5BC21D031C4FEF42E
:109270006BEC5CF0C5BC1BD0C582C5B2FED7040147
:1092800030516FD9010F10240401FE6F6BEC5CF0BC
:10929000C5BC0DD00401FC6B4DEC5CF032C4E9FFA1
:1092A00033C4EAFFEF6EC584C5B4FED7000CC58495
:1092B000C5B4FED7010C05011A510201F95D106E0B
:1092C000040E105C4DE3F9C21AF53ED9D00E316F91
:1092D0001BC530F4BDDF00093CE1070100AF39D008
:1092E00005011B511CD9EF28106E070E1016116ACC
:1092F000126A136A1B510DD9EFCF14F0156A166A62
:10930000176A1050141808E11150151805E1125091
:10931000161802E1135017181CE016D9D10E316F40
:109320001BC530F495DF05011B51FFD81B51F7D841
:10933000EF50EF2A0F011024E96E000E1120EA6EA3
:1093400000C7EFFF070E106E05011B51E8D8105043
:10935000EF1605011B2B1BC510F0CFD801E31B6BCB
:10936000120034C410F0C9D801E3000C04013451D8
:10937000DCD83451CED8EF50EF2A1024E96E000E1D
:109380001120EA6EEFCF44F7070E106E3451C1D8AA
:109390001050EF1607014451120012000401385119
:1093A0009F0805E238390F0B0F0B570F04D03839DF
:1093B0000F0B0F0B300FCFD80F0E04013815090813
:1093C00004E20F0E3815570F03D00F0E3815300F6B
:1093D000ABEF4AF007018E6B04013C5101E1000C38
:1093E000C750040B01E0010EAAD8FAE1C580C5B050
:1093F000FED7040139517BD8C5BC18D007018D6B4D
:1094000004013C5107018D5D14E204013AC4E9FFF7
:109410003BC4EAFF3A2B000E3B23EFCFFEF46BEC8C
:109420005CF0C5BC03D007018D2BEAD70701010E04
:109430008E6FC584C5B4FED707018E511200C75088
:10944000040B01E0010E7BD8FAE1C580C5B0FED760
:1094500004013D514CD8C5AC04D0C584C5B4FED779
:10946000010C0401800EFE6F6BEC5CF004013EC445
:10947000E9FF3FC4EAFF3E2B000E3F23EFCF8DF7FD
:10948000EF5003E08DC7FEF4EFD7C584C5B4FED717
:10949000000CC750040B01E0010E51D8FAE1C58061
:1094A000C5B0FED70401405122D8C5AC04D0C58454
:1094B000C5B4FED7010C0401800EFE6F6BEC5CF0AE
:1094C000040141C4F6FF412B42C4F7FF000E4223C2
:1094D00043C4F8FF43230800F5CF00F7F55003E03D
:1094E00000C7FEF4EBD7C584C5B4FED7000C39D84D
:1094F00010240401FE6F6BEF5CF0116A126A136AAC
:10950000010E105C000E1158000E1258000E135878
:109510001200EA6A2E0FE96E040EEA221200EA6ACD
:109520002F0FE96E040EEA221200080DF3CF10F09F
:10953000F4CF11F0260E1026040E11221200106E28
:109540001F0EC514101012000401000E326F070E1A
:10955000336F040112000401366F37C435F4CDEFC8
:1095600049F0E824106EE66E760E03012A6F2B6B2D
:0C95700042EC43F0E552E7CF10F012008F
:04957C00140E0301C5
:10958000B46FB56B0301020EB26F070EB36F36EC0A
:1095900027F0F00E07010215106E116A126A136AA5
:1095A000400E101805E1115003E1125001E1135073
:1095B00001E0000C0F0E0215040DF3CF8DF4040131
:1095C000F350106E116A140E105E000E115A10C086
:1095D0001CF7116A126A136AD880280E1054000E04
:1095E0001154000E1254000E135401E2000C070136
:1095F0001C5100080BE21C510301B46FB56B030151
:109600001D0EB26F070EB36F36EC27F00CC716F7BE
:109610000DC717F707010C6B0D6B140E1BD9020E4B
:109620003F6F070E406F44EC36F0F3CF18F7F4CFDE
:1096300019F70701181F191F1C51000810E21C51CF
:1096400009D91D0E3F6F070E406F44EC36F0F3CF83
:109650001AF7F4CF1BF707011A1F1B1F02D01A6B52
:109660001B6B040EF7D8180E3F6F070E406F44ECCB
:1096700036F0F3CF00F7F4CF01F70701F3501619D6
:1096800002E10151171901E0000C0401020E9D6F67
:10969000070E9E6FB2D804018E518F110CE08EC45C
:1096A000E9FF8FC4EAFF12C7EEFF13C7EEFF14C72E
:1096B000EEFF15C7EEFF90C4E9FF91C4EAFF060E66
:1096C000E3D80EC7EEFF0FC7EEFF10C7EEFF11C7BE
:1096D000EEFF92C4E9FF93C4EAFF0BC7EFFF8D5181
:1096E000126E136A07011250045D106E1350055973
:1096F000116E94C4E9FF95C4EAFF10C0EEFF11C0DB
:10970000EDFF010C0401140E8D6F0701450E926FE1
:10971000936B140E040199250701946F000E040148
:109720009A210701956F05011C2B000E1D231CC5F6
:1097300096F71DC597F70701986B400E996F640E59
:109740009A6F98C49BF79C6B9D6B00C39EF701C3F7
:109750009FF702C3A0F703C3A1F796C4E9FF97C41C
:10976000EAFF060E91D8EECFA2F7EECFA3F7EECF29
:10977000A4F7EFCFA5F70401920E9D6F070E9E6F21
:109780003CD8140E67D8920E3F6F070E406F44EC22
:1097900036F0F3CF9CF7F4CF9DF7140E0401992512
:1097A0000301C36F000E04019A210301C46F03017A
:1097B000C26B96C4E9FF97C4EAFF96C4C0F397C48E
:1097C000C1F34FEC29F0140E0301B06FB16B03012C
:1097D000920EAE6F070EAF6F7CEC26F0F36AF46A60
:1097E000120004018D519B250301CA6F000E040174
:1097F0009C210301CB6F0EEF2AF027D8020E35D83B
:10980000020E38D8020E2BD8020E39D8040E2DD8ED
:10981000040E30D8040E23D8040E31D8060E25D8F5
:10982000060E28D8060E1BD8060E29D80A0E1DD8FB
:109830000A0E20D80A0E13D80A0E03D8CDC7EFFFA0
:10984000120022D8010E44EF4CF09DC4E9FF9EC4E3
:10985000EAFF12000301416F426B0301120014D8AA
:10986000E552E750EF6E25EF4CF00ED8EFCFCDF775
:1098700025EF4CF0E6DFEF50E66E25EF4CF0E1DF30
:10988000CDC7EFFF25EF4CF0E926000EEA221200CB
:109890001C0E0301B46FB56B0301000EB26F070E0F
:1098A000B36F36EC27F006EC28F00301000EFE6FD4
:1098B000070EFF6F2FD900C710F001C711F0126A11
:1098C000136A010E101817E1115015E1125013E13F
:1098D000135011E107010451146E156A060E141895
:1098E0000AE1155008E10551166E176A040E1618A4
:1098F00001E1175001E0000C3BD9020E101809E1FC
:10990000115007E1125005E1135003E138D9EF6A15
:1099100012D02ED9010E10180AE1115008E1125090
:1099200006E1135004E1010E2AD9EF6E04D0020EB5
:1099300026D9EF6E000C030100510701185D2EE1DE
:10994000030101510701195D29E1030102510701DA
:109950001A5D24E10301035107011B5D1FE1F7C3F9
:10996000E9FFF8C3EAFF08C7EEFF09C7EEFF0AC721
:10997000EEFF0BC7EEFF0CC7EEFF0DC7EEFFF7C300
:10998000E9FFF8C3EAFF060E04D90EC7EEFF0FC7C2
:10999000EEFF10C7EEFF11C7EEFF010C000C030134
:1099A000010EAC6F37EC26F007011C6F106E116AC8
:1099B000126A136AE868101807E1115005E11250A5
:1099C00003E1135001E1000C0301CD6BCE6B1CC70A
:1099D000CCF321EC2AF0010E0701006F016B026B42
:1099E000080E036F060E046F040E056FFDC310F022
:1099F000116A126A136A010E101810E111500EE17B
:109A000012500CE113500AE1010E066F076B126948
:109A10001369146915691669176913D0020E066F68
:109A2000076BFBC3E9FFFCC3EAFFEECF12F7EECFF3
:109A300013F7EECF14F7EECF15F7EECF16F7EFCF03
:109A400017F704C308F705C309F706C30AF707C3E6
:109A50000BF708C30CF709C30DF700C30EF701C3DA
:109A60000FF702C310F703C311F77BD8EF500E199D
:109A700003010A151BE175D8010E8BD8EF500701C1
:109A80000F1903010B1512E16CD8020E82D8EF50AA
:109A90000701101903010C1509E163D8030E79D8E9
:109AA000EF500701111903010D1509E00EC318F756
:109AB0000FC319F710C31AF711C31BF709D051D8F8
:109AC000EECF18F7EECF19F7EECF1AF7EFCF1BF75F
:109AD0000301000EFE6F070EFF6F1CD81C0E030162
:109AE000C36FC46B0301060EC26F0301120EC06F79
:109AF000070EC16F4FEC29F01C0E0301B06FB16B64
:109B00000301000EAE6F070EAF6F7CEC26F0ACECDD
:109B100029F0010C39D819D8F3CFEEFF11C0EDFFB1
:109B200033D8020E36D811D8020EF3CFEBFF030E56
:109B300011C0EBFF29D8060E2CD807D8060EF3CF9C
:109B4000EBFF070E11C0EBFF1200EECF39F3EDCFA4
:109B50003AF310EC36F0F3CF10F0F4CF11F0C4EF7D
:109B60004DF0FBC3E9FFFCC3EAFF060EC9EF4DF061
:109B700006C710F007C711F0126A136A1200F9C382
:109B8000E9FFFAC3EAFF1200FEC3E9FFFFC3EAFFE1
:0A9B90001200E926000EEA2212007E
:069B9A000001FF51020A68
:109BA00025E0030A05E0010A01E01200FF2B120084
:109BB000890E0101A56FA66B0101A36BA46B0101C6
:109BC000A16FA26BEAEC2AF00101FB6F106E116A23
:109BD000126A136AE868101807E1115005E1125083
:109BE00003E1135001E112000001FF2BFBC1AEF1B4
:109BF00065EC2CF0000901E112000101060EB06FC6
:109C0000070E2ED9050EB06F070E2AD9080EB06FB9
:109C1000070E26D9070EB06F070E22D90A0EB06FB5
:109C2000070E1ED9090EB06F070E1AD90C0EB06FB1
:109C3000070E16D90B0EB06F070E12D90E0EB06FAD
:109C4000070E0ED90D0EB06F070E0AD9100EB06FA9
:109C5000070E06D90F0EB06F070EB16F84EC2CF013
:109C6000070109C710F00AC711F00907000E0A5BC7
:109C70001050111071E00101110EFC6F070EFD6F05
:109C80008ED80101000EB06F070EEAD8020EB06F39
:109C9000070EE6D8010EB06F070EE2D8040EB06FC3
:109CA000070EDED8030EB06F070EB16F84EC2CF0F8
:109CB0000701200E0119D4E10251D2E1010E03196E
:109CC000CFE10451CDE10101110EFE6F070EFF6FD0
:109CD0009FD80009C5E0FBC1A8F14AEC2BF00009B0
:109CE00003E1D7EC45F0F7D70701076B840E086F47
:109CF00006C7A9F156EC2BF005C7A9F156EC2BF0DD
:109D000008C7A9F156EC2BF007C7A9F156EC2BF0C8
:109D1000A3D8A2D8B8D822D89FD80101200EB0D895
:109D2000B2D89AD80101060EABD80101600EA8D8AE
:109D300093D800C3A9F156EC2BF001C3A9F156EC5E
:109D40002BF002C3A9F156EC2BF003C3A9F156EC9A
:109D50002BF0FCEC2BF084D7D2EF2CF00101200E7D
:109D60008FD80701216B100E215D17E2470E2125C8
:109D700003012A6F2B6B42EC43F00701226FE83896
:109D80000F0B410F01017CD80F0E07012215410F67
:109D9000010176D80701212BE6D72CEF4FF0010106
:109DA000210EB06F070EB16F84EC2CF0070121512A
:109DB0002107000924E059D82239F00B236F21072D
:109DC00054D821C710F0116A126A136AD8801E0E87
:109DD0001054000E1154000E1254000E1354E6E3FA
:109DE00023512211E66E0101FCC1E9FFFDC1EAFF2A
:109DF000FC2B000EFD23E552E750EF6ED7D70F0E78
:109E00000101EA6AFC25E96EFD51EA22EF6A1200BF
:109E10000701216B0F0E215D1EE2470E2125030174
:109E20002A6F2B6B42EC43F00701226F0101FEC148
:109E3000E9FFFFC1EAFFFE2B000EFF23EFCF23F760
:109E400007012351225D01E0000C2351225D01E056
:109E5000010C212BDFD7010C0101A96B56EF2BF070
:109E6000B16F84EC2CF0010112000101220EB06FE1
:109E7000070EB16F84EC2CF0410E0701225F120037
:109E8000A96F56EF2BF0E8DF0101010EF9DFE4DFE7
:089E9000E3DFE2DF2CEF4FF0ED
:089E980003016C6B6B816B93FD
:109EA0001FEC25F06BEC5AF0DEEC2AF006EC12F019
:109EB000160E53D9010B02E1DBEC2EF01200160E48
:109EC0004CD9010B2EE057EC28F0000922E10301E8
:109ED0006B51020B1EE103012A6B2B6B42EC43F02A
:109EE0000301006F010E39D90301016F020E35D94C
:109EF0000301026F030E31D90301036F0A690B6B73
:109F00000C6B0D6B05010F9503016B816B83C8EC26
:109F10002EF0F6EC2EF005010FA103D003016B919A
:109F20006B930701BE6B03016C51040A01E1EAD097
:109F3000070A01E1ADD0050A01E197D0010A01E16C
:109F400081D0050A39E0070A31E0050A03E0010A79
:109F500001E0F9D00301BD0EBE6F070EBF6F030114
:109F60006D0EBC6F030EBD6F65EC28F0000901E1BA
:109F7000EAD00701010EBE6FF5D810501110121073
:109F8000131003E10301020E57D0ECD8060E10188F
:109F900001E0B5D0115001E0B2D0125001E0AFD0D5
:109FA000135001E0ACD00301050E46D078EC5AF016
:109FB000000901E1C8D0C5D00401770E946F030EEB
:109FC000956F0401BD0E926F070E936F04016D0E25
:109FD000906F030E916F0401B90E8E6F070E8F6F95
:109FE000BEEC4AF000092BE00701010EBE6FBAD8A3
:109FF000101809E1115007E1125005E1135003E177
:10A000000301030E19D0AED8060E101809E1115045
:10A0100007E1125005E1135003E10301060E0CD0D5
:10A02000A1D8110E10180AE1115008E1125006E1F2
:10A03000135004E10301070E6C6F85D0BE6B06EC74
:10A0400028F07FD077C3BAF178C3BBF10101B90E14
:10A05000B86F070EB96F01016D0EB66F030EB76FC3
:10A06000DAEC2CF000096FE06CD077C3D7F078C33E
:10A07000D8F00001B90ED56F070ED66F00016D0E36
:10A08000D36F030ED46F0AEC17F000095CE059D0CF
:10A090006C6B77C310F078C311F0126A136AD88022
:10A0A000290E1054000E1154000E1254000E1354B9
:10A0B00026E304019B0E7F6F030E806F0401990E4F
:10A0C0007D6F030E7E6F0401770E7B6F030E7C6F36
:10A0D0000401790E796F030E7A6F0401BD0E776F5C
:10A0E000070E786F62EC53F0000909E0080E0701D3
:10A0F000BD5D05E1010EBE6F0301040E6C6F06EC41
:10A1000028F021D00301010EAB6F17EC26F00009F7
:10A110001AE09BC389F49CC38AF499C387F49AC359
:10A1200088F477C386F40401790E846F030E856F7B
:10A130000401836B04016D0E816F030E826FDCECF2
:10A1400053F003016C6BD7EC45F00701BE5101E001
:10A15000E8D6E3EC15F0FEEF25F003012A6F2B6B38
:10A1600042EF43F0BDC710F0116A126A136A120081
:10A170009398939A07014F6B030E4F5D0EE223D91C
:10A18000EE6AED6A20D9020E45D91DD9040E42D9D6
:10A190001AD9060E3FD94F2BEFD70401206B0501CA
:10A1A000066B076B0501086B096B12009250010BDF
:10A1B00018E008C510F039D914E18050010B1CD902
:10A1C00034D902E1000E01D0010E005D0AE0050164
:10A1D00008810701005103E00501068102D0050155
:10A1E00006919250020B1EE008C510F0126A136A25
:10A1F000020ED4D817E18050020B01E0010EFCD80A
:10A20000020ECCD802E1000E01D0010E005D0AE082
:10A21000050108830701005103E00501068302D010
:10A22000050106939250040B1EE008C510F0126A57
:10A23000136A040EB3D817E18050040B01E0010E3D
:10A24000DBD8040EABD802E1000E01D0010E005D98
:10A250000AE0050108850701005103E005010685B4
:10A2600012000501069512000701416B14C510F09C
:10A27000DCD834E012C5A8F14AEC2BF000092EE03E
:10A28000C2D8D3D80BE005010891A8D8300E8FD8DA
:10A29000CCD802E1300E01D0310EA8D8B4D8020ECD
:10A2A0007DD80CE00501089399D8310E80D8020EB4
:10A2B00075D802E1300E01D0310E98D8A4D8040E22
:10A2C0006DD80CE00501089589D8320E70D8040EBF
:10A2D00065D802E1300E01D0310E88D80701415116
:10A2E0001200F36AF46A120004012251010A0BE021
:10A2F000010A01E0120093982351E8B08A88E8B07F
:10A3000008D08A981200939A2351E8B08A8AE8A06C
:10A310008A9A120004012451050A2EE0010A25E060
:10A32000070A1CE0010A13E0030A0AE0010A01E03F
:10A3300012002551E8B08980E8B023D0899012003E
:10A340002551E8B08982E8B01CD0899212002551CD
:10A35000E8B08984E8B015D0899412002551E8B09E
:10A360008B84E8B00ED08B9412002551E8B08B821C
:10A37000E8B007D08B9212002551E8B08B80E8A09E
:10A380008B9012008A50200B01E0010EE824106E21
:10A390008A50100B01E0010E101012001016116A05
:10A3A000126A136A1050111012101310120038D8CC
:10A3B0003D0EA96F56EC2BF006C510F007C511F045
:10A3C000126A136A12004F51080DF3CFE9FFF4CF60
:10A3D000EAFF080EE926040EEA2212000701418175
:10A3E0000101780E1DD8340E10EF52F0010118D87B
:10A3F0003B0EA96F56EF2BF00701006F06C510F05A
:10A40000126A136A120008C510F009C511F0126A29
:10A41000136A1200E926000EEA22EE6AED6A1200C3
:10A42000A96F56EC2BF001011200010ECEEF51F096
:10A430000501146B0501156B0A0E03015F6F606B5C
:10A440000301000E5D6F070E5E6F19EC38F001011D
:10A45000A56BA66B0101000EA36F070EA46F7D0E06
:10A460001ED9106E116E106A10C0E6FFE66E7C0EEB
:10A4700016D9E552E7CF11F0E552E7CF10F0010110
:10A480001010A16F11C0A2F1EAEC2AF00501126FC1
:10A49000106E116A126A136AE868101805E111500B
:10A4A00003E1125001E11350120005011551020A97
:10A4B00024E0030A10E0010A01E0120012C5AEF127
:10A4C00065EC2CF000094FE0C5D802E10501146BE2
:10A4D0000501010E10D014C510F0EFD844E0E4D807
:10A4E00042E02A0EE66E920EE66E000E95D8FCEC67
:10A4F0002BF00501020E156F12000701406B12C50B
:10A50000AEF165EC2CF0000905E0A4D82CE10501C2
:10A51000146B1200050116510201F95D106E050E53
:10A52000105C1BE3F9C216F50501170710E1140EC4
:10A53000176F14C510F0C1D80AE0B6D808E0230E92
:10A54000E66E920EE66E000E67D8070140810CD8C9
:10A550000701401354D80701401340C710F0ADD88D
:10A5600002E0FCEC2BF012000701416B426B42C78A
:10A5700010F0116A126A136A010E105C000E115875
:10A58000000E1258000E135838E207014251EA6AD1
:10A590002F0FE96E040EEA22EFCF10F04251EA6A63
:10A5A0002E0FE96E040EEA22EF50105C24E042C741
:10A5B00034F4B1EC49F00701436F14C510F065D8CD
:10A5C000E4E072D8E2E00701418101016C0E72D82B
:10A5D0000101330E6FD8340E0701422501016AD8FC
:10A5E00001013D0E67D843C7A9F156EC2BF00101DC
:10A5F0003B0E60D8CAD7422BBAD741511200870E02
:10A600004ED8020802E1B9EF34F0870E48D80108AD
:10A6100002E134EF51F0000CE66E000EE66E070E1C
:10A62000E66E3BEC56F0106E050EE15E1050000E2B
:10A63000E66E070EE66E54EC56F0E552E552F3CFA7
:10A64000ACF1F4CFADF10101000EAA6F070EAB6FB4
:10A6500089EF2BF0020E0101B46FB56B0101000E02
:10A66000B26F070EB36F9EEC2CF0D2EC2CF003010E
:10A67000140E486F050E496F0301000E466F070E5A
:10A68000476F36EC37F000091200010E1016116A00
:10A69000126A136A105011101210131012000301E5
:10A6A0002A6F2B6B42EF43F012C5A8F14AEC2BF056
:10A6B00000091200A96F56EF2BF0116A126A136A93
:04A6C00045EF53F01F
:0CA6C400080E0301B46FB56B0301000E1B
:10A6D000B26F070EB36F36EC27F0080E106E18D964
:10A6E000E850EF5E15D9EF500301B46FB56B79C434
:10A6F000B2F37AC4B3F336EC27F002C72AF703C7E4
:10A700002BF70701026B036B080E0301416F426BCD
:10A710000301000E3F6F070E406F44EC36F0F3CF9D
:10A720002CF7F4CF2DF707012C1F2D1FF1D8EF5078
:10A730000301416F426B79C43FF37AC440F344ECA8
:10A7400036F0F3CF2EF7F4CF2FF707012E1F2F1F70
:10A75000040E0301416F426B03012C0E3F6F070E85
:10A76000406F44EC36F0F3CF28F7F4CF29F704011B
:10A77000000E8B6F070E8C6F96D877C4E9FF78C4F4
:10A78000EAFF00C7EFFF7DC4E9FF7EC4EAFF04C70C
:10A79000EEFF05C7EDFF7FC4E9FF80C4EAFF06C7EF
:10A7A000EEFF07C7EDFF07012A51281902E12B51DF
:10A7B000291901E0000C010C0301010EAC6F37EC0C
:10A7C00026F007012A6F106E116A126A136AE86890
:10A7D000101807E1115005E1125003E1135001E197
:10A7E0001200140E0301CD6FCE6B2AC7CCF321ECFF
:10A7F0002AF004018651106E7DD810C028F711C0D0
:10A8000029F70701016B83C400F7026B036B87C450
:10A8100004F788C405F789C406F78AC407F704015A
:10A820008651E66EE66A84C4E6FF85C4E6FF080E3C
:10A83000E66E070EE66EC0EC55F0106E060EE15E99
:10A8400010500401000E8B6F070E8C6F2CD828C798
:10A8500041F329C742F30301000E3F6F070E406F1B
:10A8600044EC36F0F3CF02F7F4CF03F786C410F0D0
:10A8700041D810C099F411C09AF40401010E986FE8
:10A8800081C496F482C497F482EC4BF028C7B0F3ED
:10A8900029C7B1F30301000EAE6F070EAF6F7CEC5A
:10A8A00026F0ACEF29F039D8040E15D8040EF3CFFA
:10A8B000EBFF050E29D8060E0ED8060EF3CFEBFFE0
:10A8C000070E22D8020E07D8020EF3CFEBFF030EBD
:10A8D00011C0EBFF1200E926000EEA22EECF39F399
:10A8E000EDCF3AF310EC36F0F3CF10F0F4CF11F0D7
:10A8F0008DEF54F0116A126A136A080E1026000ECA
:10A90000112212221322120011C0EBFF8DEF54F01E
:10A910007BC4E9FF7CC4EAFF12008BC4E9FF8CC44E
:04A92000EAFF120038
:0CA92400FF0EE3CFEAFFE552FF0EE3CF89
:10A93000E9FFE552E66AE66AD9CFE6FFDACFE6FF3D
:10A94000FC0EE124D96EFF0EE220DA6EE66AE66ABA
:10A95000E66A200EEF5C06E0090EEF5C03E0EF66AE
:10A9600003D03FD0EE50F5D72D0EEF5C03E1FF0E84
:10A97000E32A03D02B0EEF5C01E1EE502F0EEF64C3
:10A9800024D03A0EEF6021D0D890F90EE336FA0EBB
:10A99000E336FD0EDECFE3FFFE0EDDCFE3FFD89002
:10A9A000F90EE336FA0EE336D890F90EE336FA0ED6
:10A9B000E336FD0EE350DE26FE0EE350DD22300EC0
:10A9C000EE5CDE26000EDD22D9D7FF0EE3CFE8FFD6
:10A9D000E85207E0F90EE31EE32AFA0ED8B4E306C4
:10A9E000E31EE552E552E552FF0EE3CFDAFFE552F2
:10A9F000FF0EE3CFD9FFE552E1CFE9FFE2CFEAFF57
:10AA0000ED52ED52EECFF3FFEFCFF4FF1200D9CFAE
:10AA1000E6FFDACFE6FFFA0EE3CFD9FFFB0EE3CF76
:10AA2000DAFFFD0EE35209E72D0EDE6EFC0EE31E8B
:10AA3000E32AFD0ED8B4E306E31EE652E652E652E0
:10AA4000FD0EE124E76EFF0EE220E46EE652F70E03
:10AA5000E3CFE6FFF70EE3CFE6FF77EC55F0F90E14
:10AA6000E124E96EFF0EE220EA6E67EC55F00AE1A0
:10AA700064EC55F009E167EC55F008E164EC55F041
:10AA800007E108D072EC55F06DEC55F072EC55F022
:10AA90006DEC55F072EC55F0DE6AF90EE126FF0E12
:10AAA000E222FF0EE3CFDAFFE552FF0EE3CFD9FF3C
:10AAB000E552FC0EE124E96EFF0EE220EA6EEECFD5
:10AAC000F3FFEFCFF4FF1200EF380F0B1200EF503F
:10AAD0000F0B02E1EE52D8841200EF380F0B300F4B
:10AAE000DE6E1200EE500F0B300FDE6E1200FC0E09
:10AAF000E3CFE9FFFD0EE3CFEAFF100EE66EEE6A4C
:10AB0000EE6AEF6AD890FD0EE336FE0EE336ED36C0
:10AB1000ED36EF36FF0EE30609E098EC55F0EE5205
:10AB200098EC55F0EE5298EC55F0EDD7E56E12002A
:10AB3000030EEF24E8B6EF6E300EEF24E8BEEF6EA2
:02AB4000000C07
:0EAB4200FB0EE3CFF6FFFC0EE3CFF7FFFD0E98
:10AB5000E3CFF8FFFE0EE3CFE9FFFF0EE3CFEAFFFE
:10AB6000F90EE35003E1FA0EE35009E0F90EE306B3
:10AB700002E2FA0EE3060900F550EE5CF1E0120085
:10AB8000D9CFE6FFDACFE6FFFA0EE3CFD9FFFB0E0F
:10AB9000E3CFDAFFFC0EE3CFE9FFFD0EE3CFEAFFE0
:10ABA000E9CFF3FFEACFF4FFF80EE35003E1F90E2B
:10ABB000E35008E0F80EE30602E2F90EE306DECF0A
:10ABC000EEFFF2D7FF0EE3CFDAFFE552FF0EE3CF41
:10ABD000D9FFE5521200FE0EE3CFE9FFFF0EE3CFEF
:10ABE000EAFFE9CFF3FFEACFF4FFFB0EE35003E106
:10ABF000FC0EE35009E0FB0EE30602E2FC0EE30666
:10AC0000FD0EE350EE6EF1D71200D9CFE6FFDACF9A
:10AC1000E6FFFA0EE3CFD9FFFB0EE3CFDAFFFC0E1F
:10AC2000E3CFE9FFFD0EE3CFEAFFDE50EF5C02E188
:10AC3000EE66FBD7F36EFF0EE3CFDAFFE552FF0EB1
:10AC4000E3CFD9FFE552F3501200FB0EE3CFF6FF3E
:10AC5000FC0EE3CFF7FFFD0EE3CFF8FFFE0EE3CFD0
:10AC6000E9FFFF0EE3CFEAFF0900F550EF5C02E1D8
:10AC7000EE66FAD71200FB0EE3CFF6FFFC0EE3CF31
:10AC8000F7FFFD0EE3CFF8FFFE0EE3CFE9FFFF0E67
:10AC9000E3CFEAFFE9CFF3FFEACFF4FF0900F5CFF6
:10ACA000EFFFEE66FBD71200FE0EE3CFE9FFFF0ECB
:10ACB000E3CFEAFFF36AF46AEE5203E0F34AF42AC0
:10ACC000FBD71200D9CFE6FFDACFE6FFFA0EE3CFCB
:10ACD000D9FFFB0EE3CFDAFFFC0EE3CFE9FFFD0E59
:10ACE000E3CFEAFFE9CFF3FFEACFF4FFF80EE3503A
:10ACF00003E1F90EE3500BE0F80EE30602E2F90E71
:10AD0000E306DECFEFFFEE66F1D7DD52EFD7FF0EA1
:10AD1000E3CFDAFFE552FF0EE3CFD9FFE552120091
:10AD2000FE0EE3CFE9FFFF0EE3CFEAFFE9CFF3FF2B
:10AD3000EACFF4FF610EEF5C05E67B0EEF5C02E705
:0AAD4000DF0EEF16EE52F6E11200EE
:06AD4A00B0C4FBF404019B
:10AD5000FA6B0401080EF96F3EEF5CF0B2C4A4F781
:10AD6000B3C4A5F7C750040B01E0010EE0D8FAE127
:10AD7000C580C5B0FED7A1B6010CB1C4FDF4DCD8C6
:10AD800001E0010CC750040B01E0010ED0D8FAE13C
:10AD9000C5BC19D0A5C7FDF4CFD801E0010CC75040
:10ADA000040B01E0010EC3D8FAE1A4C7FDF4C4D836
:10ADB00001E0010CC750040B01E0010EB8D8FAE124
:10ADC000C5AC000C020C020CB5C4B2F4B6C4B3F4AA
:10ADD000B4C4B1F4C3DF0701086FE85005E173D8CC
:10ADE0000701086FE85002E008511200C750040B39
:10ADF00001E0010E9CD8FAE1C580C5B0FED7A1B62E
:10AE0000010C0401B4290401FD6F96D801E0010C86
:10AE1000C750040B01E0010E8AD8FAE1C5AC000C62
:10AE2000020CC750040B01E0010E81D8FAE1B7C44F
:10AE3000FDF482D801E0010CC750040B01E0010EC3
:10AE400076D8FAE1C5AC000C020CC750040B01E047
:10AE5000010E6DD8FAE1C584C5B4FED7000C04011B
:10AE6000010EFC6F4DEC5CF0C95012000401FC6B4C
:10AE70004DEC5CF0C584C5B4FED7000CB9C4B5F484
:10AE8000BAC4B6F4B8C4B4F49FDF0701006FE85049
:10AE900018E10401BD51BD07000910E00401010ED5
:10AEA000FC6F4DEC5CF00401BBC4E9FFBCC4EAFFDD
:10AEB000BB2B000EBC23C9CFEFFFEBD7D7DF0701B9
:10AEC000006F00511200C750040B01E0010E2FD893
:10AED000FAE1C584C5B4FED7A1B6010C000CC75079
:10AEE000040B01E0010E23D8FAE1C580C5B0FED7FE
:10AEF000A1B6010CBEC4FDF41FD801E0010CC7507F
:10AF0000040B01E0010E13D8FAE1A1B6010CC5BC97
:10AF100003D00701A86B03D00701040EA86FC584F6
:10AF2000C5B4FED7A1B6010C0701A8511200106EDE
:10AF30001F0EC5141010120064EC5CF00009120022
:10AF400012000701406B416B446BE2C4C3FBE3C4D6
:10AF5000C4FBFAEC23F00701456F400E426F0B0172
:10AF6000420EAF6F070EB06F0B01000EAD6F070EF4
:10AF7000AE6FE2C4E9FFE3C4EAFFEF500B01AC6F30
:10AF8000BFEC21F00701436F442B476B6C0E005D53
:10AF900008E10151750A02E0050A1EE1010E476F42
:10AFA0001BD06D0E005D18E145C710F0116A98D8EE
:10AFB00005E0ADD86F0A02E1010E476FA8D86C0A10
:10AFC0000BE1010E476FE2C4E9FFE3C4EAFF090E9B
:10AFD000E926000EEA22EF88475116E145C7DBF368
:10AFE00042510301D96FDA6B000ED927070EDA231D
:10AFF0000301000ED76F070ED86F62EC06F0F35016
:10B0000007014013F45041134351A7E170D8020ED9
:10B0100086D801E012006BD8040E81D804E07DECE4
:10B0200043F0D1EF43F063D8080E79D802E0D2EFB5
:10B0300043F05DD8100E73D802E015EF44F057D8F6
:10B04000106A010E11164CD802E0FFEF44F04FD801
:10B05000106A200E111644D802E031EF45F047D8AF
:10B06000106A080E11163CD802E0CCEF40F03FD831
:10B07000106A100E111634D802E047EC41F01200AD
:10B080003DD8020EE926000EEA22EFCF00F736D8AF
:10B09000030EE926000EEA22EFCF01F72FD8EECFFC
:10B0A00002F7EDCF03F7E8C404F7E9C405F7E8C4F5
:10B0B000E9FFE9C4EAFFEF6AE6C4C3FBE7C4C4FBE7
:10B0C000FAEC23F00701066F0301000EDC6F070E98
:10B0D000DD6FC9EC0DF002C7F3FF03C7F4FF1200E8
:10B0E000126A136A1050111012101310120040C788
:10B0F00010F041C711F0126A136A1200E6C4E9FFAA
:10B10000E7C4EAFF040EE926000EEA2212004251CB
:10B11000EA6A000FE96E070EEA22EF5012001016DD
:06B12000116A70EF58F007
:0AB126000D0A507265737320616E0C
:10B1300079206B657920666F7220436F6E66696750
:10B1400075726174696F6E206D656E752E000D0AE3
:10B1500052756E6E696E67204170706C69636174C0
:10B16000696F6E2C20495020616464726573733A74
:10B170002000444843502F476C65616E696E672E0E
:10B180002E2E000D0A0D0A0D4D6F6474726F6E69DC
:10B190007820576562205365727665720D0A0D0A34
:10B1A00009313A204368616E676520426F617264BD
:10B1B0002073657269616C206E756D6265722E0D0B
:10B1C0000A09323A204368616E67652064656661EA
:10B1D000756C7420495020616464726573732E0D20
:10B1E0000A09333A204368616E67652064656661C9
:10B1F000756C74206761746577617920616464722D
:10B200006573732E0D0A09343A204368616E6765D1
:10B210002064656661756C74207375626E65742058
:10B220006D61736B2E0D0A09353A20456E61626CB3
:10B23000652044484350202620495020476C6561D2
:10B240006E696E672E0D0A09363A20446973616291
:10B250006C652044484350202620495020476C65A7
:10B26000616E696E672E0D0A09373A20446F776E5A
:10B270006C6F61642046696C652053797374656DE9
:10B2800020496D6167652E0D0A09383A20536176B1
:10B2900065202620517569742E0D0A0D0A456E74BD
:10B2A00065722061206D656E752063686F696365E6
:10B2B0002028312D38293A20000D0A496E76616C1C
:10B2C000696420696E70757420726563656976655E
:10B2D00064202D20496E7075742069676E6F7265E9
:10B2E000642E0D0A507265737320616E79206B6550
:10B2F0007920746F20636F6E74696E75652E2E2EC3
:08B300000D0A001B5B324A003C
:08B30800040EAC6E100EAB6EDA
:10B310009D9A9D981200AC8AAB88AB8E9D8A0201E3
:10B32000F58F1200AC9AAB98AB9E9D9A9D98020146
:10B33000F59F12000201D36BD3C2D1F2D3C2D2F275
:10B34000D96BD9C2D7F2D9C2D8F21200060EAB140B
:10B3500002E0AB98AB889EAA17D00201DA51D95D02
:10B360000FE0D751EA6AD525E96ED651EA22AECF71
:10B37000EFFFD72BDA51D75D01E1D76BD92BEBD794
:10B38000F589AE50A86EE7D712000201D35103E150
:10B39000F5939D981200D25198D8EF50AD6ED22BF4
:10B3A000D451D25D01E1D26BD30712000201F5B393
:10B3B00012D0D35110E0D25188D8EFCF04F7D22B5E
:10B3C000D451D25D01E1D26BD307F29E04C7ADFF29
:10B3D000F5839D88F28E12000201D9510EE0D851FA
:10B3E000EA6AD525E96ED651EA22EFCFA4F7D82B29
:10B3F000DA51D85D01E1D86BD9070701A4511200D9
:10B400000201D451D35D03E1D7EC45F0F9D7F29EA8
:10B41000F5B305D0F2C4ADFFF5839D880AD0D151B4
:10B4200054D8F2C4EFFFD12BD451D15D01E1D16BDF
:10B43000D32BF28E12000401F3519F0805E2F33979
:10B440000F0B0F0B570F04D0F3390F0B0F0B300FEF
:10B450000401F26FD5DF0F0E0401F315090804E2B1
:10B460000F0EF315570F03D00F0EF315300F040115
:10B47000F26F00EF5AF00401F4C4E9FFF5C4EAFFEB
:10B48000F42B000EF523EFCF08F7EF5006E008C7C6
:10B49000F2F4B6DFD7EC45F0EED712000401F6C4A3
:10B4A000F6FFF62BF7C4F7FF000EF723F8C4F8FFFA
:10B4B000F8230800F5CF00F7F55006E000C7F2F4D6
:10B4C0009FDFD7EC45F0EAD71200EA6ACF25E96E94
:06B4D000D051EA22120037
:0AB4D60004019F6BA069A169A2693F
:10B4E000A369A469A569A66BA76BA86BA96B1200D9
:10B4F00004019F5130E10301270EF96F070EFA6F27
:10B5000003011D0EF76F070EF86F48EC4CF00009B1
:10B5100031E027C710F0116A126A136A1050111037
:10B520001210131015E11DC7A0F41EC7A1F41FC708
:10B53000A2F420C7A3F421C7A4F422C7A5F423C70B
:10B54000A6F424C7A7F425C7A8F426C7A9F4010CBC
:10B550000401010E9F6F0301FD6B03011D0EFB6FC4
:10B56000070EFC6FCFEC4CF0000903E004019F6B69
:10B57000010C000C010CAAC4E9FFABC4EAFFEECF3A
:10B5800023F7EECF24F7EECF25F7EFCF26F7030111
:10B59000010EFD6F03011D0EFB6F070EFC6FCFEF59
:10B5A0004CF0ACC4E9FFADC4EAFF0401A651EE18AB
:10B5B00008E1A751EE1805E1A851EE1802E1A951E2
:10B5C000EE1814E003010E510401A65D20E1030111
:10B5D0000F510401A75D1BE1030110510401A85D97
:10B5E00016E1030111510401A95D11E1AEC4E9FFA7
:10B5F000AFC4EAFFA0C4EEFFA1C4EEFFA2C4EEFFF9
:10B60000A3C4EEFFA4C4EEFFA5C4EEFF010C000C22
:10B610000401EA6B120012000201DF6BDFC2DDF2EF
:10B62000DFC2DEF2E56BE5C2E3F2E5C2E4F212004E
:10B630000201E5510EE0E451EA6AE125E96EE251CA
:10B64000EA22EFCF00F7E42BE651E45D01E1E46B81
:10B65000E5070701005112000201DD51EA6ADB250E
:10B66000E96EDC51EA22EBC4EFFFDD2BE051DD5D3A
:10B6700001E1DD6BDF2B12000401EC519F0805E2B4
:10B68000EC390F0B0F0B570F04D0EC390F0B0F0BCE
:10B69000300F0401EB6FE0DF0F0E0401EC15090819
:10B6A00004E20F0EEC15570F03D00F0EEC15300F00
:10B6B0000401EB6F2CEF5BF00401EDC4E9FFEEC475
:10B6C000EAFFED2B000EEE23EFCF00F7EF5006E080
:10B6D00000C7EBF4C1DFD7EC45F0EED71200040150
:10B6E000EFC4F6FFEF2BF0C4F7FF000EF023F1C418
:10B6F000F8FFF1230800F5CF00F7F55006E000C78A
:0CB70000EBF4AADFD7EC45F0EAD712000A
:04B70C005458540039
:10B7100048544D00434C4100435353004A530000EA
:10B7200047494600434749004A5047004A415200B2
:10B7300057415600545854005A5458005A4854001F
:10B740005A434C005A4353005A4A530048545450E9
:10B750002F312E3020323030204F4B00436F6E742B
:10B76000656E742D747970653A2000436F6E746550
:10B770006E742D456E636F64696E673A20677A69EF
:10B78000700D0A00457870697265733A20300D0AB1
:10B790000043616368652D436F6E74726F6C3A206D
:10B7A0006D61782D6167653D3330302C206D757388
:10B7B000742D726576616C69646174650D0A004769
:10B7C000455400494E4445582E48544D004C4F476F
:07B7D000494E2E43474900DA
:08B7D8002A0EF66E080EF76E52
:10B7E000000EF86E04010900F550DD6F0900F550F8
:10B7F000DE6F03E1DD6701D03DD00900F550D86F61
:10B800000900F550D96F0900F550DA6F09000900F9
:10B81000F550E96E0900F550EA6E090009000900CB
:10B82000F550DB6F0900F550DC6F09000900F6CF19
:10B83000DFF4F7CFE0F4F8CFE1F4D8C4F6FFD9C4D1
:10B84000F7FFDAC4F8FF0401DB5302E1DC5307E041
:10B850000900F550EE6EDB07F8E2DC07F9D7DFC42C
:10B86000F6FFE0C4F7FFE1C4F8FF0401DD07000EB6
:06B87000DE5BBFD71200F1
:0AB87600C6BEC69E12003F0EC716A4
:10B88000C66AC56A0401F951C612FA51C7129486F4
:10B890009488C68AFBC4C8FF1200C586C7B003D00F
:10B8A000D7EC45F0FBD7C5B6FED70401FC5102E04A
:10B8B000000E01D0010EE8B0C58AE8A0C59AC5887F
:10B8C000C5B8FED7C9501200FDC4C9FFC6BEFF0CE3
:10B8D000C7B0FED7000CFEC4C9FFC6BE010CC7B07E
:10B8E000FED7C750040B01E0010E106E1F0EC514E9
:06B8F0001010F7E1000C4E
:0AB8F6004142434445464748494A91
:10B900004B4C4D4E4F505152535455565758595A0F
:10B910006162636465666768696A6B6C6D6E6F709F
:10B920007172737475767778797A30313233343551
:07B93000363738392B2F00D8
:08B938000B01FE51FE0700099E
:10B9400007E007010D0E8D6F8D51F6E08D07FCD7D6
:10B9500012000B01FF51FF07000908E0080EE66E18
:0EB96000F7EC5CF0E552D7EC45F0F3D712009F
:02B96E0063680C
:10B9700065636B65640064697361626C6564003C57
:10B98000212D2D002D2D3E006F6E006F6666004E3E
:0FB990006F7420496D706C656D656E7465640031
:10B9A000036A026A100EE76ED89006360736023632
:10B9B00003360B50025C0C50035805E30B50025E3B
:0CB9C0000C50035A062AE72EF0D71200A4
:04B9CC000201F96B10
:10B9D000FA6BFB6BFC6BFD6BFE6B580ED66E9E0E0E
:0EB9E000D76E010ED56ED58EF284F28A12005B
:02B9EE00FF0E4A
:10B9F000E350246E480E01D04C0EE76EE72EFED7C2
:0EBA0000E76AE72EFED7242EF7D700001200CB
:02BA0E005633AD
:10BA10002E313000415554484F52495A4154494FF4
:0ABA20004E3A2042415349432000F2
:06BA2A001CEE00F02CEE02
:10BA300000F0F86A0F9CECEC5BF0F1EC45F0FDD700
:02BA40001200F2
:0EBA42000501066B076B086B096B1200120002
:0EBA500000EE00F00D0EEE6AEA62FDD7120065
:02BA5E0056325E
:04BA60002E3531004E
:02BA64000004DC
:0ABA6600F69000DF9000C39000ABE3
:0EBA700090008B90006A90002B90000E9000CA
:02BA7E00FF00C7
:02BA80000000C4
:02BA82000000C2
:02BA84000000C0
:0ABA8600039000F98F00E58F00DC4B
:10BA90008F00CC8F00C28F00F98F00B78F009E8F70
:10BAA00000918F00039000039000F98F00E58F0054
:0FBAB000DC8F00CC8F006A8F00438F00E28E0086
:01BABF007C0A
:10BAC0002424247D72737475767778797A7B2424A4
:10BAD00024242424243E3F404142434445464748D1
:10BAE000494A4B4C4D4E4F50515253545556572482
:10BAF000242424242458595A5B5C5D5E5F60616293
:10BB0000636465666768696A6B6C6D6E6F707100FF
:10BB10001492000F92000A9200059200009200FB1E
:10BB20009100F69100EA9100D29100C29100B89183
:10BB300000B191009B91008691006B910060910093
:09BB4000489100119100089100E8
:03BB4900020014E3
:04BB4C000100FF00F5
:02BB5000FF00F4
:02BB5200FFFFF3
:06BB5400BE0F00BB0F0054
:020000040030CA
:0100010026D8
:0100020006F7
:010003000CF0
:010005008377
:010006008178
:010008000FE8
:010009008076
:01000A000FE6
:01000B008074
:01000C000FE4
:01000D0000F2
:0200000400F00A
:100000000A0100010004A3000000FF0000000A0133
:10001000000104012803010A0100010A010001078F
:10002000010700FFFFFFFFFFFFFF000000000000CF
:1000300000032E000061646D696E0000000070779F
:10004000000000000000004D58424F415244202063
:10005000202020202020000A0100016BD300000096
:10006000000001000201000000000000000000008C
:100070000000350050005000000000006CD300006C
:100080000000000000000000000000000000000070
:100090000000000000000000000000000000000060
:1000A0000000000000000000000000000000000050
:1000B0000000000000000000000000000000000040
:1000C0000000000000000000000000000000000030
:1000D0000000000000000000000000000000000020
:1000E0000000000000000000000000000000000010
:1000F0000000000000000000000000000000000000
:100100006464000000000000000000000000000027
:0C0110006DD3016ED300FFFF1122339964
:00000001FF
